:100000000C9450020C9478020C9478020C94391CD5
:100010000C9478020C9478020C9478020C9473047B
:100020000C9478020C9478020C9478020C94780268
:100030000C9478020C9478020C9478020C94780258
:100040000C9482280C9478020C94F5040C94CF0440
:100050000C9478020C9478020C9478020C94780238
:100060000C9427050C947802FB2BBA2CCC2C202D59
:10007000242D672D9A2DE42DE82DEF2DF82D0F2E30
:10008000892F982FA92FAF2F24306030C030F53042
:100090001C3144317F319B31B431B431E831F93115
:1000A000FC310132063209324368616E6765204BCC
:1000B000657920547970653F004357204B6579205E
:1000C000547970652073657421004357205374611F
:1000D00072742044656C61790043572054582D3E5A
:1000E00052582044656C6179004368616E676520F1
:1000F000435720546F6E650053696465746F6E6575
:1001000020736574210043617272696572207365A2
:1001100074210050545420746F20636F6E666972AE
:100120006D2E2000536574204357205258204246BC
:100130004F004361727269657220736574210050CB
:10014000545420746F20636F6E6669726D2E2000A8
:1001500054756E6520746F206265737420536967EF
:100160006E616C00536574207468652042464F00D0
:100170005365742043617272696572206E6F7700F7
:1001800043616C6962726174696F6E20736574217A
:100190000070726573732050545420746F20736123
:1001A00076650053657420746F205A65726F2D62F6
:1001B0006561742C005365742043616C69627261DF
:1001C00074696F6E3F0045786974204D656E753FA8
:1001D000005365747570204F6E3F005365747570E1
:1001E000204F66663F00534452204D6F6465204F98
:1001F00066663F00534452204D6F6465204F6E3F4A
:10020000005753505220426561636F6E0057535040
:10021000523A0050545420746F2053656E64004D60
:10022000656D6F7279204B657965720056464F2077
:10023000546F204368616E6E656C3F004368616E69
:100240006E656C20546F2056464F3F004154542039
:100250004F6E3F00415454204368616E67653F0014
:100260004946205368696674204F6E3F0049462016
:100270005368696674204368616E67653F00536523
:100280006C656374204D6F64653F0053656C6563F6
:10029000742056464F20413F0053656C65637420BF
:1002A00056464F20423F00507265737320746F2092
:1002B000636F6E6669726D0048616D2062616E6485
:1002C0000047656E6572616C0042616E6420536523
:1002D0006C6563743F00507265737320746F207394
:1002E0006574005365742054756E65205374657091
:1002F0003F004469616C3A467265712054756E65C1
:10030000004469616C3A53656C6563742054657888
:100310007400534452204D4F44450053504B204DE0
:100320004F44450053706C6974204F6E3F0053502A
:1003300054204F6E00535054204F66660053706C2B
:100340006974204F66663F00456D70747920646162
:10035000746100524954204F66663F005249542050
:100360004F6E3F00496E697420454550726F6D2E87
:100370002E2E00D5F3CCDEEBA4ACED90F8EAA294DF
:10038000E1CDD2DA94A290C5AC2E2C3F22212F28A9
:1003900029263A3B3D2B2D5F2740237E5B5D5E1F68
:1003A0000F0703010010181C1E00000000000000D1
:1003B0000000000000000000000024484A381042FD
:1003C0003C4020473A442C283E464D3430183241B8
:1003D00036494B4C00435720537065656420736564
:1003E0007421004357205370656564207365742140
:1003F0000053696465746F6E6520736574212043D2
:1004000041540053696465746F6E6520736574218F
:1004100020434154004175746F4B657920457869DC
:10042000742F4341540000000000240027002A00DC
:100430005458204F46463F005458204F4E005458C1
:10044000204F4646005458204F4E3F000000000009
:10045000250028002B0002000000002300260029B0
:10046000000404040404040404020202020202035D
:100470000303030303010204081020408001020467
:1004800008102001020408102000000008000201EA
:100490000000030407000000000000000000933982
:1004A00011241FBECFEFD8E0DEBFCDBF12E0A0E029
:1004B000B1E0ECE5F6E702C005900D92AA34B10771
:1004C000D9F726E0AAE4B2E001C01D92A539B2072F
:1004D000E1F712E0C0E5D2E004C02197FE010E94DE
:1004E000CD3ACF34D107C9F70E94CC280C942C3BCD
:1004F0000C940000CF92DF92EF92FF920F931F9324
:10050000CF93DF936C017A018B01C0E0D0E0CE1570
:10051000DF0581F0D8016D918D01D601ED91FC913F
:100520000190F081E02DC6010995892B11F02196EB
:10053000EECF7E01C701DF91CF911F910F91FF9008
:10054000EF90DF90CF900895FC01538D448D252FBF
:1005500030E0842F90E0821B930B541710F0CF965D
:10056000089501970895FC01918D828D981761F08F
:10057000828DDF01A80FB11D5D968C91928D9F5FDA
:100580009F73928F90E008958FEF9FEF0895FC0185
:10059000918D828D981731F0828DE80FF11D858D38
:1005A00090E008958FEF9FEF0895FC01918D228DCB
:1005B000892F90E0805C9F4F821B91098F73992750
:1005C000089581EE95E00E94D50221E0892B09F47F
:1005D00020E0822F0895FC01848DDF01A80FB11D5A
:1005E000A35ABF4F2C91848D90E001968F73992769
:1005F000848FA689B7892C93A089B1898C91837047
:1006000080648C93938D848D981306C00288F3893F
:10061000E02D80818F7D80830895EF92FF920F936C
:100620001F93CF93DF93EC0181E0888F9B8D8C8D9E
:10063000981305C0E889F989808185FD26C0F62ECA
:100640000B8D10E00F5F1F4F0F731127E02E8C8D65
:10065000E8120CC00FB607FCFACFE889F98980814F
:1006600085FFF5CFCE010E94EB02F1CF8B8DFE010D
:10067000E80FF11DE35AFF4FF0829FB7F8940B8FFC
:10068000EA89FB89808180620AC09FB7F894EE896D
:10069000FF896083E889F989808183708064808321
:1006A0009FBF81E090E0DF91CF911F910F91FF906C
:1006B000EF900895CF93DF93EC01888D8823C9F0E4
:1006C000EA89FB89808185FD05C0A889B9898C915B
:1006D00086FD0FC00FB607FCF5CF808185FFF2CFF6
:1006E000A889B9898C9185FFEDCFCE010E94EB02DC
:1006F000E7CFDF91CF91089580E090E0892B29F03A
:100700000E94E10281110C940000089585ED809310
:10071000BC008091BC0084FDFCCF1092A20508951E
:1007200040915C04262F30E0240F311D2132310529
:10073000DCF42091A2052430C9F4FC0180E090E0B3
:10074000861758F430915C042191DC01A45CBB4F06
:10075000A30FB11D2C930196F3CF80915C04680F19
:1007600060935C0480E0089581E0089582E008953C
:10077000089508950895E091210480912004E817D8
:1007800030F4F0E0E050FC4F808190E008958FEF6E
:100790009FEF08959091210480912004981750F4C0
:1007A000E92FF0E0E050FC4F208130E09F5F909314
:1007B000210402C02FEF3FEFC9010895809120046A
:1007C00090E020912104821B91090895CF92DF923D
:1007D000EF92FF920F931F93CF93DF937C01CB0196
:1007E0008A012091A305222389F0EB016B01C40E3D
:1007F000D51ECC15DD0569F06991D701ED91FC910D
:100800000190F081E02DC7010995F3CF642F0E947C
:100810009003C801DF91CF911F910F91FF90EF904E
:10082000DF90CF900895CF93DF931F92CDB7DEB7BF
:1008300069832091A3052223D1F02091C60520329F
:1008400040F021E030E0FC013383228380E090E03F
:1008500015C08091A405E82FF0E0EB55FA4F99817F
:1008600090838F5F8093A4058093C60505C061E0E7
:10087000CE0101960E94900381E090E00F90DF91FD
:10088000CF910895089580E090E008950E94F53A90
:1008900090916301891324C0E6E5F4E0E4919FEFB1
:1008A00090936301E130B9F098F0E230C9F490918F
:1008B00070009D7F9093700091E09093B0009091B4
:1008C000B100987F94609093B1001092B30008C07B
:1008D00010926E0005C090916F009D7F90936F0005
:1008E00060E00C94A4251F920F920FB60F92112472
:1008F0002F933F934F935F936F937F938F939F9328
:10090000AF93BF93EF93FF938091DD059091DE0548
:10091000A091DF05B091E005892B8A2B8B2B51F13B
:100920009091DA05E091DB05F091DC058081892763
:1009300080838091DD059091DE05A091DF05B09167
:10094000E005181619061A061B06C4F48091DD0589
:100950009091DE05A091DF05B091E0050197A10916
:10096000B1098093DD059093DE05A093DF05B09378
:10097000E00504C0809163010E944804FF91EF915B
:10098000BF91AF919F918F917F916F915F914F91A7
:100990003F912F910F900FBE0F901F9018951F92AF
:1009A0000F920FB60F9211242F933F934F935F93A3
:1009B0006F937F938F939F93AF93BF93EF93FF9327
:1009C00081EE95E00E94EB02FF91EF91BF91AF9114
:1009D0009F918F917F916F915F914F913F912F9157
:1009E0000F900FBE0F901F9018951F920F920FB689
:1009F0000F9211242F938F939F93EF93FF93E09186
:100A0000F105F091F2058081E091F705F091F8058C
:100A100082FD12C090818091FA058F5F8F732091C3
:100A2000FB05821751F0E091FA05F0E0EF51FA4F23
:100A3000958F8093FA0501C08081FF91EF919F917E
:100A40008F912F910F900FBE0F901F9018951F92AE
:100A50000F920FB60F9211242F933F934F935F93F2
:100A60006F937F938F939F93AF93BF93EF93FF9376
:100A70008091B900887F803609F49CC068F588327F
:100A800009F45BC090F4803109F454C038F4882331
:100A900009F4F6C0883009F44DC0F6C0883109F475
:100AA0004CC0803209F45DC0EFC0803409F468C0E6
:100AB00048F4803309F455C0883309F0E5C08093C9
:100AC000A005D8C0803509F44FC0883509F45DC051
:100AD000883409F0D9C0D6C0883909F4C7C0A8F451
:100AE000883709F467C038F4883609F463C0803762
:100AF00009F460C0C9C0883809F4B8C0803909F465
:100B00005FC0803809F0C0C05BC0803B09F486C07C
:100B100038F4803A09F466C0883A09F47FC0B4C05A
:100B2000803C09F4A7C0883C09F4A4C0883B09F4C0
:100B30008AC0AAC080917D0510C090919F058091C8
:100B40009E05981770F5E0919F0581E08E0F8093C8
:100B50009F05F0E0E258FA4F80818093BB0085EC5E
:100B600086C08093A0058EC0E0919F0581E08E0F26
:100B700080939F058091BB00F0E0E258FA4F80839C
:100B800090919F0580919E056EC0E0919F0581E048
:100B90008E0F80939F058091BB00F0E0E258FA4FE2
:100BA00080838091A10581116DC081E080937C05D7
:100BB00084EA61C083E08093A20510927E04CFCFC7
:100BC00080917E04803208F051C0E0917E0481E083
:100BD0008E0F80937E048091BB00F0E0E25AFB4FC1
:100BE0008083BDCF85EC8093BC001092A2058091DC
:100BF0007E04803230F4E0917E04F0E0E25AFB4F54
:100C0000108260917E0470E0E0912404F09125044C
:100C10008EE594E0099510927E0436C084E08093BE
:100C2000A20510925D0410925C04E0912204F09100
:100C30002304099580915C04811105C081E08093B3
:100C40005C0410923C04E0915D0481E08E0F80937F
:100C50005D04F0E0E45CFB4F80818093BB009091E9
:100C60005D0480915C04981708F479CF85E880933F
:100C7000BC000AC085EC8093BC001092A20504C0A1
:100C80001092A0050E948603FF91EF91BF91AF9152
:100C90009F918F917F916F915F914F913F912F9194
:100CA0000F900FBE0F901F9018958091FE0281301B
:100CB00029F41092FE026BE173E011C081E0809391
:100CC000FE0280910503813011F41092050380919A
:100CD000DC03813011F41092DC0362E173E080E008
:100CE0000E9490126EEF72E082EF90E00E94030C7F
:100CF0006091D6057091D7058091D8059091D9055E
:100D00000E94FA170E94250E1092C80508952F928E
:100D10003F924F925F926F927F928F929F92AF928B
:100D2000BF92CF92DF92EF92FF920F931F93CF93D8
:100D3000DF93CDB7DEB72E970FB6F894DEBF0FBEA8
:100D4000CDBF80910403282F30E0A8E2B4E0EDEDA0
:100D5000F3E0AF014D5D5340421753071CF49191EE
:100D60009D93F7CF10920403E8E2F4E020E030E036
:100D7000082E000C990B0397281739070CF0F5C2C1
:100D800041914935B9F440814835A1F44181483653
:100D900089F4A901485D5B4F5A834983DA011396B0
:100DA0008C91813051F461E0E981FA8184810E9463
:100DB000D00EB5C22F5F3F4FDFCF823041F4F90133
:100DC000E45DFB4F80819181A281B3815CC183305E
:100DD000B1F58091D8029EEF980F923018F08656A8
:100DE0008230C8F4C090D605D090D705E090D805E1
:100DF000F090D905C701B6010E94111A082F87FD8E
:100E00000AC00E944D0F282F30E040E050E0C7019B
:100E1000B6010E94D919A981BA8114968C918130AA
:100E200011F041E001C04FEF6091D6057091D705F8
:100E30008091D8059091D9050E940D1B70C2843015
:100E400019F40E94F90E6BC2853029F48AE090E013
:100E50000E94EA1264C2863029F481E090E00E9488
:100E6000B7125DC2873029F481E090E00E94EA2445
:100E700056C2883019F40E94550651C2893081F457
:100E8000909162018091C705903119F4809581702D
:100E900004C08695817091E089270E940B253FC28E
:100EA0008A3031F4E981FA8184818093970237C2D4
:100EB0008B3041F481E090919A02911180E080930F
:100EC0009A022DC28C3051F4F901E45DFB4F808110
:100ED0009181909399028093980221C28D3009F0FC
:100EE00042C0A981BA8114960C91149710E015960E
:100EF000CC901597D12C16968C90BAE08B9E400121
:100F000011241A830983092C000CAA08BB088091BC
:100F10000403811104C2E981FA81AF01FF0F660B5E
:100F2000770B8EE60E94341DE980FA80FFEFEF1AFE
:100F3000FF0A29813A812C593E4FD9018C910E9498
:100F40001F28AC01990F660B770B88E70E94341DB0
:100F5000CE14DF040CF47801C501B4010E943C28D2
:100F6000FA82E982D4CF8E3009F4FFC1803109F0D2
:100F700093C08091D6059091D705A091D805B091E6
:100F8000D90589839A83AB83BC83A0912701B09153
:100F90002801BE83AD838090250190902601809129
:100FA000230190912401F901E45DFB4FB081BB87DF
:100FB00021812C872280338000E010E09C0140E0FA
:100FC00050E02F83388749875A87092C000CAA08DC
:100FD000BB084D815E81041715070CF050C08AE7ED
:100FE00091E09E878D87AD85BE858D91BE87AD874B
:100FF0000E94F31BE5E8F1E02D853E85E217F3073B
:1010000091F7CB84DC847101412C512C32014814BE
:1010100059046A047B0468F5C701B6010E94FA17F7
:1010200088E590E00E942F0C9E878D87FC0124E0CC
:10103000F595E7952A95E1F7E659FE4F80810E94E4
:10104000F31B4D855E854F70552746595E4FDA017B
:101050008C910E94F31BBFEF4B1A5B0A6B0A7B0A51
:101060002F81388549855A85C20ED31EE41EF51E90
:10107000CECF81E00E94F21C0F5F1F4FAACF898163
:101080009A81AB81BC818093D6059093D705A093BC
:10109000D805B093D90543C18F3029F5A981BA810C
:1010A00014968C91149790E09093280180932701D7
:1010B00015968C91159790E09093270480932604C1
:1010C00016968C91169790E09093260180932501B7
:1010D00017968C91B4E18B9FC00111249093240149
:1010E000809323011CC1813131F4E981FA8184812B
:1010F0008093FC0214C1823151F4A981BA81149603
:101100008C9190E09093200180931F0108C183315E
:10111000A9F4E981FA8194819093600281E09111B0
:1011200001C080E08093220180912101913011F46F
:101130008F7E01C0806180932101F1C0853121F44F
:1011400081E080939B02EBC08F3109F065C0F9010B
:10115000E45DFB4F60807180A981BA8116968C9006
:10116000169717960C9110E0EAE7F1E0FA83E9830D
:1011700095E8E92E91E0F92EA981BA818D91BA8383
:10118000A9830E94F31BE981FA81EE16FF06A1F7FD
:10119000282D30E0215031093A832983C12CD12CEC
:1011A0007601912CA12CB12CC814D904EA04FB04BB
:1011B00078F50834110551F589819A81860D971DBE
:1011C0000E942D0C582EE82FF0E00735110581F014
:1011D00084E0F595E7958A95E1F7E659FE4F808121
:1011E0000E94F31BE52DEF70F0E0E659FE4F808181
:1011F0000E94F31B3FEFC31AD30AE30AF30A4981A3
:101200005A81415051095A834983CECFC601D6CF66
:1012100081E00E94F21C83C0803209F03FC0F901D6
:10122000E45DFB4F00811181A981BA811696EC9093
:101230001697F12C17964C91179750E015966C91D4
:101240001597808190E0860F911D8E0D9F1D481788
:101250005907D9F46D01C801885294405C01A21A63
:10126000B30AC601E981FA818E1B9F0B8E159F057B
:1012700074F4D60118966C91C5018C0D9D1D0E94C9
:101280002B0CBFEFCB1ADB0AECCF0EEF1FEFA80140
:1012900060E070E08EE60E94341D41C08A3491F413
:1012A000F901E45DFB4F408151816281738186E7E2
:1012B0000E945D1D4AE450E060E070E087E60E9415
:1012C0005D1D2DC0853511F08F3549F5F901E45DBF
:1012D000FB4F40815181628173814C365844654493
:1012E0007945E9F48F3529F40E9454240C940000C8
:1012F00016C01A82198289819A818F5B9F4F0E9442
:101300002D0C682F89819A810E942B0C29813A81AA
:101310002F5F3F4F3A8329832032310561F7609177
:10132000D6057091D7058091D8059091D9050E9476
:10133000FA170E94250E2E960FB6F894DEBF0FBE48
:10134000CDBFDF91CF911F910F91FF90EF90DF9074
:10135000CF90BF90AF909F908F907F906F905F9055
:101360004F903F902F900C942D112E960FB6F8941D
:10137000DEBF0FBECDBFDF91CF911F910F91FF90C8
:10138000EF90DF90CF90BF90AF909F908F907F9025
:101390006F905F904F903F902F9008952F923F92C3
:1013A0004F925F926F927F928F929F92AF92BF9275
:1013B000CF92DF92EF92FF920F931F93CF93DF9321
:1013C000CDB7DEB728970FB6F894DEBF0FBECDBFFE
:1013D000A82E60E084EF91E00E949319B12CE12CDB
:1013E000F12CDD24D39400E010E0AAE02A2E312C69
:1013F000412C512C0E94490D892B09F0DFC021E0BE
:10140000D212B2C0ECE9F2E02EE111922A95E9F78E
:101410000431110538F06EE172E08CE992E00E942F
:10142000153B9EC0BE016B5F7F4FC801880F991F9F
:10143000880F991F8A589D4F0E94DD0B8D819E81D8
:10144000AF81B885AC01BD01FDE1769567955795F3
:101450004795FA95D1F7B42EBF718D839E83AF83E4
:10146000B8870A30110554F586E0809F6001819F9E
:10147000D00C1124C6018A539D4F0E942D0C83303D
:10148000E9F43601E9E36E1AEDEF7E0A6CE9862E87
:1014900062E0962EF4E3CF1AFDEFDF0AC3010E944B
:1014A0002D0CF40181934F01FFEF6F1A7F0A6C142A
:1014B0007D04A1F78AE38093A10224C067E372E070
:1014C0008CE992E00E94153B093011051CF420E3E1
:1014D00020939E02B8016F5F7F4F072E000C880B90
:1014E000990B2AE04AEB52E00E94D7396AEB72E08E
:1014F0008CE992E00E94013B64E272E08CE992E0A8
:101500000E94013B6D817E818F8198854CE9C42EBC
:1015100042E0D42E5FE0852E912C61157105810586
:10152000910589F094012B7F2830310511F42EE2CA
:101530000BC0A20191010E948C3A605DF6016787A1
:10154000B901CA0103C020E2F6012787E1E08E1A43
:101550009108F1E0CF1AD10825E082169104E9F64E
:101560008CE992E00E946C110E94920C0097E1F0CD
:101570001CF48FEF9FEF02C081E090E0E80EF91EAF
:101580008DEFE8168FEFF8062CF417FD0FC0015011
:1015900011090CC0E4E0EE16F10434F00431110539
:1015A0002CF40F5F1F4F02C0D12C04C0E12CF12C92
:1015B000DD24D39480E00E94F51F1CCF0431110577
:1015C00008F048C0F1E0AF1218C08D819E81AF8154
:1015D000B885895B9B40A109B10987349B47A34922
:1015E000B340C0F561E08B2D0E94D00E6D817E81ED
:1015F0008F8198850E94FA172DC00E944D0F40914F
:10160000D6055091D7056091D8057091D9057F71A5
:1016100090E0A0E0B0E02DE1880F991FAA1FBB1F4A
:101620002A95D1F7842B952BA62BB72B89839A83E8
:10163000AB83BC83C801880F991F880F991FBE0117
:101640006F5F7F4F8A589D4F0E94650B87E292E043
:101650000E946C1160E084EF91E00E9493190E9457
:1016600065111092C80528960FB6F894DEBF0FBE1C
:10167000CDBFDF91CF911F910F91FF90EF90DF9041
:10168000CF90BF90AF909F908F907F906F905F9022
:101690004F903F902F90089580E090E00C944F245D
:1016A000CF938EE00E941F28C1E0853F91400CF44B
:1016B000C0E08FE00E941F28853F914014F480E035
:1016C00001C082E08C0FCF910895AF92BF92CF926C
:1016D000DF92EF92FF920F931F93CF93DF9300D08F
:1016E000CDB7DEB78B016B0124E0C20ED11C7B01AC
:1016F0005C01A61AB70AC5018E0D9F1DF701619105
:101700007F019A838983CE0101960E94DA1BEC1433
:10171000FD0489F7C8010F900F90DF91CF911F91C1
:101720000F91FF90EF90DF90CF90BF90AF90089512
:10173000EF92FF920F931F93CF93DF9300D0CDB71B
:10174000DEB78C017B01FB0160819A838983CE0126
:1017500001960E94DA1BF70161810F5F1F4F1A8308
:101760000983CE0101960E94DA1BC7010F900F90EA
:10177000DF91CF911F910F91FF90EF9008950F93FC
:101780001F93CF93DF938C01EB010E94323A888341
:10179000C80101960E94323A8983CE01DF91CF9130
:1017A0001F910F910895CF93DF93EB010E94323A7E
:1017B0008883CE01DF91CF910895CF92DF92EF928F
:1017C000FF920F931F93CF93DF93EB017B0124E0F4
:1017D000E20EF11C8B016C01C61AD70AC601800FFC
:1017E000911F0E94323AF80181938F01EE15FF0597
:1017F000A9F7CE01DF91CF911F910F91FF90EF904C
:10180000DF90CF9008950F931F93CF93DF9300D075
:10181000CDB7DEB78B01FB0160819A838983CE014E
:1018200001960E94DA1BC8010F900F90DF91CF91B3
:101830001F910F910895CF93DF9380934801C4E4E3
:10184000D1E089910E94F31B81E0CF34D807C9F71A
:10185000DF91CF9108950C943A3A0C94323A1816CD
:10186000190694F4BC0191E09093A30598E5909338
:10187000C5051092A4051092C6058EE796E00E9459
:10188000130481E00E9422258091A2058111FCCFE2
:1018900081E08093A2058093A1059FEF9093A0051E
:1018A00010929F0510929E0580937D0580917D0585
:1018B000806B80937D0580917C05813061F410926E
:1018C0007C0580917D058093BB008091BC0083FDE9
:1018D000F8CF85EC01C085EE8093BC008091A20515
:1018E0008130E1F380919F05811103C090919F05A4
:1018F00001C091E0AEE7B5E0E0E0F4E080E08917F8
:1019000021F02D9121938F5FFACF109221048093C3
:101910002004882321F08EE796E00C94CA0380E02F
:1019200090E008958F929F92AF92BF92CF92DF92F4
:10193000EF92FF920F931F93CF930E9476284B0153
:101940005C01E12CF12C0E947628DC01CB01881986
:101950009909AA09BB09C297A105B10508F058C0A9
:101960000E94500BC82FC82ED12C0091420110911B
:101970004301C016D10631F061E070E080E090E0F4
:101980000E943C280E94500BC813DDCFC016D10620
:10199000D1F20115110519F4C230B9F511C00230A8
:1019A000110519F4C33091F40BC00330110519F47B
:1019B000C13091F405C001301105A1F4C11109C075
:1019C00081E0E81AF10801151105F9F0013011055F
:1019D00019F4C33079F40BC00330110519F4C23087
:1019E00049F405C00230110529F4C11103C08FEF7D
:1019F000E81AF80AD0924301C092420161E070E017
:101A000080E090E00E943C289ECFC13099F7EFCF54
:101A1000C701CF911F910F91FF90EF90DF90CF9072
:101A2000BF90AF909F908F900895CF93DF9380E108
:101A30000E941F28D82FC92F80E10E941F288035BF
:101A4000910514F18D2F9C2F97FD03969595879501
:101A500095958795E4E8F4E02281222369F040819E
:101A600050E08417950744F0418150E0481759072A
:101A70001CF0822F90E00AC0339624E0E43BF2078A
:101A800059F78FEF9FEF02C088E790E0DF91CF9189
:101A9000089580E10E941F2821E030E08135910502
:101AA00014F020E030E0C9010895CF93C62F909143
:101AB0007B0521E02093A3059093C5051092A40512
:101AC0001092C605682F8EE796E00E9413046C2FD3
:101AD0008EE796E00E94130481E0CF910C942225BA
:101AE0008F929F92AF92BF92CF92DF92EF92FF922E
:101AF0001F93CF93DF93CDB7DEB728970FB6F89437
:101B0000DEBF0FBECDBF182F6A017B01DB01CA010A
:101B10008052914AA740B10981329449A747B64003
:101B200050F081E090E001C0880F1A95EAF790919B
:101B30000A01892B71C060910601709107018091A3
:101B4000080190910901A70196010E948C3A460173
:101B5000570188249924E0EFAE2289288A288B280F
:101B600049F09695879577956795F694E794D7947D
:101B7000C794EDCFE7E0660F771F881F991FEA959E
:101B8000D1F749015A01F7E0880C991CAA1CBB1C2B
:101B9000FA95D1F722E0921AA108B108A70196019F
:101BA0000E948C3A820E931EA41EB51ED982CA8250
:101BB000AB829C828D82CC24DD24EFE0EE22FF24D8
:101BC000A4E0CC0CDD1CEE1CFF1CAA95D1F7C62AA4
:101BD000D72AE82AF92AEE827F836887812F880F27
:101BE000880F880FBE016F5F7F4F865D0E947E2544
:101BF000E12FF0E0EB57FE4F60816C6080E1810FD8
:101C00000E94550D81E090E001C0880F1A95EAF717
:101C1000809590910A01892380930A0160910A01BD
:101C200083E00E94550D28960FB6F894DEBF0FBED4
:101C3000CDBFDF91CF911F91FF90EF90DF90CF90BC
:101C4000BF90AF909F908F9008958091D90281119D
:101C500009C04091650250916602609167027091DF
:101C6000680208C040916102509162026091630273
:101C70007091640280919A02882369F08091060332
:101C8000811109C08091980290919902092E000C4F
:101C9000AA0BBB0B03C080E090E0DC01840F951F12
:101CA000A61FB71F2091FE02222349F020910603B0
:101CB000211105C040E050E060E070E002C0AC01DE
:101CC000BD0180E00C94700D10922104109220044C
:101CD0001092A4051092C6051092A20581E080938F
:101CE000A10510927C0561E082E10E94A42561E0DB
:101CF00083E10E94A425E9EBF0E080818E7F808360
:101D000080818D7F808388E48093B80085E4809310
:101D1000BC0088EB93E0909323048093220489EB2A
:101D200093E0909325048093240460E085E90E9469
:101D3000550D60910A0183E00E94550D60E887EB24
:101D40000E94550DEAE3F1E012828FE0838380E880
:101D50008483BF018AE10E947E2560E281EB0E94BC
:101D6000550D6AE371E082E20E947E2560EA81EB14
:101D70000E94550D8091690290916A02A0916B02B8
:101D8000B0916C0280549F48A84DBB4C80930601D3
:101D900090930701A0930801B09309010C94250EBC
:101DA000843011F481E003C0853021F482E0809317
:101DB000D90208951092D902833011F481E013C042
:101DC0006130A1F4811112C081E04091D60550919B
:101DD000D7056091D8057091D905413856496849B1
:101DE000710508F480E08093E70208951092E702FD
:101DF00008950E945424809162018431F9F480E1B5
:101E00008093620180915A0190915B01A0915C01E5
:101E1000B0915D018093D6059093D705A093D80526
:101E2000B093D9058093000390930103A09302031C
:101E3000B093030360E08091D4051EC084E18093D9
:101E4000620180915E0190915F01A0916001B0916B
:101E500061018093D6059093D705A093D805B093E0
:101E6000D9058093000390930103A0930203B093DC
:101E7000030360E08091D5050E94D00E0E942619D0
:101E80006091D6057091D7058091D8059091D905BC
:101E90000E94FA171092C80508958091D902811105
:101EA00006C08091E702811106C082E0089581306A
:101EB00021F085E0089583E0089584E00895CF93AC
:101EC000DF9380932D01605D60933301C9E2D1E01F
:101ED00089910E94F31B81E0C733D807C9F7DF91CE
:101EE000CF91089590910001981731F080930001EF
:101EF000682F80E30C945F0F089561E08091620188
:101F0000803109F460E08091D904681729F060936A
:101F1000D90486E70E945F0F4091D6055091D705FE
:101F20006091D8057091D9058091D5049091D6041F
:101F3000A091D704B091D80484179507A607B707D6
:101F400059F04093D5045093D6046093D70470930E
:101F5000D80483E60E945D1D0E944D0F9091D40429
:101F6000891731F08093D404682F83E60E945F0FB5
:101F700080910803811170C18091C805811181E0B1
:101F80000E94720F40915A0150915B0160915C0177
:101F900070915D018091D0049091D104A091D20400
:101FA000B091D30484179507A607B70759F040935B
:101FB000D0045093D1046093D2047093D30481E68B
:101FC0000E945D1D6091D4058091CF04861729F091
:101FD0006093CF0481E60E945F0F40915E015091B3
:101FE0005F0160916001709161018091CB049091DB
:101FF000CC04A091CD04B091CE0484179507A60718
:10200000B70759F04093CB045093CC046093CD04B0
:102010007093CE0482E60E945D1D6091D50580918B
:10202000CA04861729F06093CA0482E60E945F0FF3
:102030006091C7058091C904861729F06093C9048F
:102040008CE60E945F0F609105038091C80486179B
:1020500029F06093C80482E70E945F0F40918004DA
:102060005091810460918204709183048091C40432
:102070009091C504A091C604B091C7048417950738
:10208000A607B70759F04093C4045093C504609362
:10209000C6047093C70482E70E945D1D6091060329
:1020A0008091C304861729F06093C30484E70E94DB
:1020B0005F0F6091C7058091C904861729F060936E
:1020C000C9048CE60E945F0F6091DC038091C2041A
:1020D00090E0262F062E000C330B8217930729F071
:1020E0006093C20483E70E945F0F6091C90561702D
:1020F0008091C104681729F06093C10488E70E94A9
:102100005F0F6091FC028091C004861729F06093F4
:10211000C0048EE60E945F0F6091FD028091BF04B3
:10212000861729F06093BF0480E70E945F0F4091FB
:1021300002015091030160910401709105018091A9
:10214000BB049091BC04A091BD04B091BE0484175F
:102150009507A607B70759F04093BB045093BC04FA
:102160006093BD047093BE0484E70E94341D6091A7
:10217000600280913901861729F0609339018BE65E
:102180000E945F0F40911F01509120018091B9047E
:102190009091BA048417950749F05093BA0440937C
:1021A000B90460E070E083E70E94341D40911D0196
:1021B00080913801841741F04093380150E060E08D
:1021C00070E089E70E94341D40911E018091370123
:1021D000841741F04093370150E060E070E085E6FD
:1021E0000E94341D409197028091B804841741F0F9
:1021F0004093B80450E060E070E086E60E94341D31
:1022000060919A028091B704861729F06093B70411
:1022100089E60E945F0F4091980250919902809147
:10222000B5049091B6048417950759F05093B604FD
:102230004093B504052E000C660B770B89E60E94CF
:10224000341D6091FE028091B404861729F06093DA
:10225000B4048AE60C945F0F089580E090E00C943B
:102260007D0F95E18902A001112443595D4F20E0C3
:1022700030E0FB019191BF01911106C0682F082E3B
:10228000000C770B90E20AC0FA01E20FF31F908373
:102290002F5F3F4F2031310561F7F0CFFA01E20F98
:1022A000F31F90832F5F3F4F24313105B9F79B0116
:1022B0002F5F3F4F95E1929FF001939FF00D112406
:1022C000E359FD4F10820C94061D6AEF71E080E027
:1022D0000E9431110C942D11BC0180E00C9431113D
:1022E0002EE1ECE9F2E0DF01322F1D923A95E9F799
:1022F000EAEBF2E0DF011D922A95E9F72AE0AF014F
:102300000E94E63942E050E06AEB72E08CE992E02C
:102310000E941C3B6AE372E08CE992E00E94013B60
:1023200043E050E06CEB72E08CE992E00E941C3BD1
:102330006AE372E08CE992E00E94013B43E050E0E6
:102340006FEB72E08CE992E00E941C3B8CE992E01A
:102350000C946C112F923F924F925F926F927F92EA
:102360008F929F92AF92BF92CF92DF92EF92FF92A5
:102370000F931F93CF93DF9300D01F92CDB7DEB79B
:102380005C017B836A833A011901480160E08CE2B9
:1023900091E00E9493198AE0A816B10484F46CE3DA
:1023A00072E08AEB92E00E94153BB7018AEB92E063
:1023B0000E94013B6AEB72E081E00E94311191E0E2
:1023C000998300E010E0442455244C185D080E94D5
:1023D000490D892B09F088C00E94920C009729F4BE
:1023E0008981813009F07BC006C0181619061CF4DB
:1023F00081E090E002C08FEF9FEF080F191F0415D6
:10240000150544F48A819B81681679067CF4881945
:1024100099090AC0C016D1065CF48A819B81821595
:10242000930524F4880D991D9B838A8300E010E0B6
:10243000B7018AEB92E00E94153B9BE0A916B1041C
:1024400059F4EA81FB81EE0FFF1FEE0FFF1FE654E8
:10245000FD4F8EE3808313C065E272E08AEB92E069
:102460000E94013B4AE06CE972E08A819B810E94F4
:10247000CC396CE972E08AEB92E00E94013B8AEB76
:1024800092E00E946C1191E0A916B10429F48A81AE
:102490009B810E940F2623C082E0A816B10441F060
:1024A00095E0A916B104D9F49A819093970206C0D9
:1024B0008A819B81909399028093980282E0809315
:1024C000C8050E942D116091D6057091D7058091A5
:1024D000D8059091D9050E94FA170E94250E80E038
:1024E0000E94F51F198273CF8A819B810F900F90F4
:1024F0000F90DF91CF911F910F91FF90EF90DF90A0
:10250000CF90BF90AF909F908F907F906F905F9093
:102510004F903F902F9008958AEF91E00C946C11AA
:10252000CF93DF93CDB7DEB765970FB6F894DEBFD4
:102530000FBECDBFAB01DE01119620E030E0BD0142
:10254000FA01E20FF31FE491ED93EE2329F02F5FE0
:102550003F4F25313105A1F70E94311165960FB625
:10256000F894DEBF0FBECDBFDF91CF9108952091CB
:102570000503892B51F4213019F463E573E002C09F
:102580006CE573E080E00C949012211114C08091EE
:10259000D6059091D705A091D805B091D90521E035
:1025A000209305038093800490938104A093820478
:1025B000B093830402C00E9426191092C8050895A2
:1025C00068E473E080E00E94901260E080ED97E0A4
:1025D0000C9493192091DC03892B51F4211103C031
:1025E00064E273E002C06DE373E080E00C9490124B
:1025F000213029F41092DC0365E373E00BC081E025
:102600008093DC0380910503813011F4109205035F
:102610006EE273E080E00E9490121092C805089567
:102620008F929F92AF92BF92CF92DF92EF92FF92E2
:102630000F931F93CF93DF9300D0CDB7DEB769E63A
:1026400072E080E090E00E94DD0B65E672E088E0D9
:1026500090E00E94DD0B6AE571E080E190E00E946D
:10266000DD0B6EE571E084E190E00E94DD0B62E03D
:1026700071E088E190E00E94DD0B6FE171E08CE198
:1026800090E00E94BF0B88E093E00E942D0C8935FA
:1026900061F489E093E00E942D0C883531F48AE0E2
:1026A00093E00E942D0C883601F164E673E081E02E
:1026B0000E94901200E410E060E0C8010E942B0C20
:1026C0000F5F1F4F011524E01207B1F769E588E09D
:1026D00093E00E942B0C68E589E093E00E942B0CAC
:1026E00068E68AE093E00E942B0C8BE093E00E9466
:1026F0002D0C843029F064E08BE093E00E942B0CD9
:102700008FE390E00E942D0C90EF980F913E08F01F
:1027100080E680937B0580E490E00E942D0C83315D
:1027200059F561E672E08CEF90E00E94DD0B64EDFC
:1027300075E080E091E00E94D30B65ED75E081E0EB
:1027400091E00E94D30B6DE171E082E091E00E9484
:10275000D30B6EE171E083E091E00E94D30B60E661
:1027600072E086E691E00E94D30B80916002833094
:10277000C8F01092600216C063E180E490E00E940D
:102780002B0C00E010E0C8010E942D0C682FC8013E
:102790008F5B9F4F0E942B0C0F5F1F4F0032110564
:1027A00091F7BFCF90916002911103C01092220166
:1027B0000CC081E08093220180912101913011F4BD
:1027C0008F7E01C08061809321016CE572E088E614
:1027D00091E00E94D30B6FEF72E089E691E00E94D6
:1027E000D30B63E175E08AE691E00E94D30BE4E845
:1027F000EE2EE4E0FE2E0CE810E0C8010E942D0C45
:10280000F7018083C80101960E942D0CF701818396
:10281000C80102960E942D0CF70182830D5F1F4FA5
:10282000F3E0EF0EF11C0C3B110539F78CE093E05F
:102830000E942D0C893531F48DE093E00E942D0C1F
:1028400080935F0262E175E084E091E00E94D30B27
:1028500068ED72E085E091E00E94D30BF12CE12C51
:1028600080911205F81658F51A82198224E0F29E1A
:1028700080011124BE016F5F7F4FC8018A5F9E4FA8
:102880000E94BF0B89819A81F801E651FB4F918329
:1028900080830297863D964D08F4E394BE016F5FF6
:1028A0007F4FC801885F9E4F0E94BF0BF801E65121
:1028B000FB4F89819A8193838283F394D1CF909146
:1028C000D8022CEF290F203640F0983630F48823B8
:1028D00021F084E08E1508F47EC082E08093D80257
:1028E0008AE08093120582E197E09093EB04809355
:1028F000EA0480ED97E09093ED048093EC048CEA79
:102900009DE09093EF048093EE0488ED9EE0909319
:10291000F1048093F00487EE94E19093F3048093A4
:10292000F20487EF94E19093F5048093F40488E532
:102930009BE19093F7048093F60484E89CE19093E4
:10294000F9048093F80484E797E29093FB04809362
:10295000FA0486EA97E29093FD048093FC0480EBEE
:1029600096E39093FF048093FE048EE098E39093A7
:1029700001058093000584E996E490930305809314
:10298000020588EF96E4909305058093040588E09E
:1029900092E590930705809306058AEC93E5909362
:1029A0000905809308058AE391E690930B058093CF
:1029B0000A058EE991E690930D0580930C0580E65B
:1029C0009DE690930F0580930E0584E094E7909325
:1029D0001105809310056CEF72E086E591E00E948E
:1029E000D30B08EE12E067E5C62EDD24D394B12C9C
:1029F00078EEE72E73E0F72EC6010E942D0C982F7B
:102A000092959695969593708F73282F30E091301C
:102A100029F4EAE08E9FC001112412C0923029F4FB
:102A2000F4E68F9FC00111240BC0933041F42E9D1A
:102A3000C0012F9D900D3E9D900D112401C0C90134
:102A4000A0E0B0E0F80181939193A193B1938F013D
:102A50000197A109B10980369A4EA105B10508F484
:102A6000B3942FEFC21AD20A4CE5C41641E0D40643
:102A700019F684E08B15E0F18AE090E0A0E0B0E088
:102A80008093E8029093E902A093EA02B093EB02EC
:102A900082E390E0A0E0B0E08093EC029093ED023E
:102AA000A093EE02B093EF0284E690E0A0E0B0E0E5
:102AB0008093F0029093F102A093F202B093F3029C
:102AC00084EF91E0A0E0B0E08093F4029093F502EF
:102AD000A093F602B093F70288EE93E0A0E0B0E096
:102AE0008093F8029093F902A093FA02B093FB024C
:102AF0008091FC02811103C083E08093FC028CE58D
:102B000091E00E942D0C182F8DE591E00E942D0C74
:102B1000212F237030E0322F2227282B30931905E4
:102B2000209318058EE591E00E942D0C212F2C702A
:102B300090E4299F90011124282B309317052093AE
:102B400016058FE591E00E942D0C212F2073E0E106
:102B50002E9F90011124282B3093210520932005CE
:102B600080E691E00E942D0C107CF4E01F9F900104
:102B70001124282B30931F0520931E0581E691E038
:102B80000E942D0C182F82E691E00E942D0C212F1F
:102B9000237030E0322F2227282B309325052093F5
:102BA000240583E691E00E942D0C212F2C7040E437
:102BB000249F90011124282B309323052093220574
:102BC00084E691E00E942D0C212F207390E1299F33
:102BD00090011124282B30931D0520931C0585E6B8
:102BE00091E00E942D0C107CE4E01E9F90011124C6
:102BF000282B30931B0520931A0587E691E00E944D
:102C00002D0C8093010190915C0297FF17C0282F33
:102C10002F73FAE02F9F9001112486FF03C0319596
:102C20002195310930935E0220935D0287FD04C037
:102C300081E08093010102C01092010196FF10C053
:102C400068E972E08BE691E00E94BF0B81E0209181
:102C5000980230919902232B09F480E080939A0224
:102C600069EE74E080EF90E00E94D30B8091E9045C
:102C700080FF10C068EE74E081EF90E00E94D30BFB
:102C80008091E90481FF06C06EEF72E082EF90E070
:102C90000E94D30B64EE74E083EF90E00E94DD0BA2
:102CA000209118053091190580911605909117050E
:102CB0002817390754F0109219051092180582E36D
:102CC00090E0909317058093160520911C05309194
:102CD0001D0580911A0590911B052817390764F08E
:102CE00083E390E090931D0580931C058CE291E0B6
:102CF00090931B0580931A052091200530912105A2
:102D000080911E0590911F052817390764F08DE208
:102D100091E0909321058093200588E592E09093BF
:102D20001F0580931E052091240530912505809173
:102D30002205909123052817390764F089E592E070
:102D4000909325058093240580E293E090932305DA
:102D50008093220580911D0181508A3F18F08CE3F9
:102D600080931D018091D405823018F482E0809315
:102D7000D4058091D505823018F483E08093D50581
:102D80008091650290916602A0916702B0916802FD
:102D900080549449A84AB109813E9E42A105B105DB
:102DA00060F080EE93EAA8EAB0E080936502909329
:102DB0006602A0936702B0936802809161029091CD
:102DC0006202A0916302B091640280549449A84ABF
:102DD000B109813E9E42A105B10560F080EE93EA03
:102DE000A8EAB0E08093610290936202A09363022C
:102DF000B093640280915A0190915B01A0915C01B3
:102E0000B0915D01805E9746A543B109813E964A27
:102E1000A04EB14078F080EB99E1ADE6B0E0809350
:102E20005A0190935B01A0935C01B0935D0182E035
:102E30008093D40580915E0190915F01A091600123
:102E4000B0916101805E9746A543B109813E964AE3
:102E5000A04EB14078F080E799EEA7EDB0E0809306
:102E60005E0190935F01A0936001B093610183E0E4
:102E70008093D50580915A0190915B01A0915C01EE
:102E8000B0915D018093D0059093D105A093D205B8
:102E9000B093D30580915E0190915F01A091600194
:102EA000B09161018093CB059093CC05A093CD05A3
:102EB000B093CE058091D4058093CF058091D50540
:102EC0008093CA058091020190910301A0910401B1
:102ED000B091050184569109A109B1098D36974039
:102EE000A105B10560F080E293E0A0E0B0E080933E
:102EF000020190930301A0930401B0930501809116
:102F00001F01909120010A978F3D934030F084E695
:102F100090E09093200180931F0180900201909097
:102F20000301A0900401B0900501C501B4016C52E9
:102F30007140810991096D3BE2E07E0781059105B1
:102F400028F0109215051092140513C022E3C22E2A
:102F5000D12CE12CF12CA70196010E948C3A2093F0
:102F60001505C501B401A70196010E948C3A609332
:102F700014050F900F90DF91CF911F910F91FF904B
:102F8000EF90DF90CF90BF90AF909F908F9008957B
:102F900061342FE6720720E4820721E0920710F0E7
:102FA00060E008C060382FE9720725ED82079105BF
:102FB00030F061E085E00E94A42560E00AC0613C39
:102FC0007F4C8A46910550F060E085E00E94A42580
:102FD00061E084E00E94A42560E009C060E085E033
:102FE0000E94A42560E084E00E94A42561E083E0C3
:102FF0000C94A4254F925F926F927F928F929F9232
:10300000AF92BF92CF92DF92EF92FF92E091FC02DB
:1030100024E0E29FF0011124EC51FD4FC080D180EB
:10302000E280F380A70196010E948C3ACA01B9019F
:10303000A70196010E94483A4B015C010E94C81703
:103040009091D902911109C040906502509066029A
:10305000609067027090680208C0409061025090D2
:103060006202609063027090640280919A02E09123
:103070000603882359F0E11109C02091980230918C
:103080009902A901330F660B770B03C040E050E0B3
:10309000BA01440E551E661E771E8091E9046091A8
:1030A000FE0280FF14C02091E80430E0662321F086
:1030B000E11102C02F503109923031F0911109C055
:1030C0004091E702442329F02E51310902C020E04B
:1030D00030E0E11107C0C090970244E6C49E600151
:1030E000112402C0C12CD12C74E6729FA001739FE1
:1030F000500D1124C40ED51E0D2C000CEE08FF0837
:1031000087FF08C0F094E094D094C094C11CD11CF7
:10311000E11CF11C662309F448C0E11146C090E0AF
:1031200095958795959587958370813019F424013D
:10313000350119C0823039F4C501B40120E836E9FF
:1031400048E950E008C0833059F4C501B40120E4D7
:1031500032E44FE050E00E948C3A2B013C0103C066
:10316000412C512C3201B501A401405F524561450B
:103170007D4F4C0D5D1D6E1D7F1D82E00E94700D08
:103180004091E4045091E5046091E6047091E704F5
:10319000405F524561457D4F4C0D5D1D6E1D7F1D8D
:1031A000440D551D661D771D39C0913031F09111C8
:1031B0001EC08091E70281111AC0D501C401885355
:1031C0009740AA4FBD4FAC01BD01440D551D661D72
:1031D000771D4C0D5D1D6E1D7F1D82E00E94700DE0
:1031E000B701A601485357406A4F7D4F17C0B5013C
:1031F000A401445B5C49684A7C4F4419550966093F
:1032000077094C0D5D1D6E1D7F1D82E00E94700DC3
:10321000B701A601445B5C49684A7C4F81E00E948B
:10322000700D8092D6059092D705A092D805B092E5
:10323000D905FF90EF90DF90CF90BF90AF909F9017
:103240008F907F906F905F904F90089580910503CD
:10325000882371F0109205036091800470918104BD
:1032600080918204909183040E94FA170C942D118E
:1032700008951092060360E087E00E94A4250E9452
:10328000250E80910503882349F06091E004709138
:10329000E1048091E2049091E30441C08091DC0359
:1032A0008130A9F5809162018431B9F480E1809385
:1032B000620180915A0190915B01A0915C01B091F3
:1032C0005D018093D6059093D705A093D805B09360
:1032D000D90560E08091D40518C08031C1F484E143
:1032E0008093620180915E0190915F01A0916001E5
:1032F000B09161018093D6059093D705A093D8052E
:10330000B093D90560E08091D5050E94D00E609100
:10331000D6057091D7058091D8059091D9050E9466
:10332000FA170C942D11CF92DF92EF92FF920F9328
:103330001F93CF936C01C62F0E9476286093DC0404
:103340007093DD048093DE049093DF04E12CF12C74
:103350000E9476280091DC041091DD042091DE04A7
:103360003091DF04DC01CB01801B910BA20BB30B6E
:10337000C816D906EA06FB0660F0C43041F484E1C1
:103380000E941F288132934034F481E00AC08C2FC0
:1033900005C080E006C00E94291E83E00E94F51F40
:1033A000D7CFCF911F910F91FF90EF90DF90CF90EB
:1033B0000895CF92DF92EF92FF920F93CF93DF9316
:1033C00000D000D0CDB7DEB707FD1FC069017A017C
:1033D000DC01CB01BF712DE1CC0CDD1CEE1CFF1C10
:1033E0002A95D1F78C299D29AE29BF2989839A83F3
:1033F000AB83BC8324E00202C0011124BE016F5FD5
:103400007F4F825D9E4F0E94650B0F900F900F9033
:103410000F90DF91CF910F91FF90EF90DF90CF90C1
:103420000895CF92DF92EF92FF9228EE33E040E0D2
:1034300050E00E948C3A90911205EAEEF4E080E0B0
:103440008917B9F0608171816B01E12CF12C2C1589
:103450003D054E055F0550F0628173816B01E12CE3
:10346000F12C2C153D054E055F0520F08F5F34963D
:10347000E7CF8FEFFF90EF90DF90CF900895CF933D
:10348000DF93D82FC62F8091D8028436D0F0809158
:103490000503882349F06091800470918104809134
:1034A00082049091830408C06091D6057091D7057D
:1034B0008091D8059091D9050E94111A8F3F09F487
:1034C000A9C08091C90580FD04C061E087E00E9429
:1034D000A42581E080930603809105038823C9F029
:1034E0008091D6059091D705A091D805B091D905C6
:1034F0008093E0049093E104A093E204B093E3048A
:103500006091800470918104809182049091830481
:1035100043C08091DC038130B9F50E94542480912E
:1035200062018431B9F480E18093620180915A0193
:1035300090915B01A0915C01B0915D018093D605F3
:103540009093D705A093D805B093D90560E08091FA
:10355000D40518C08031C1F484E180936201809168
:103560005E0190915F01A0916001B0916101809333
:10357000D6059093D705A093D805B093D90560E000
:103580008091D5050E94D00E6091D6057091D70527
:103590008091D8059091D9050E94FA170E94250EB6
:1035A000D13091F540E050E0BA0180E00E94700D0A
:1035B00040E050E0BA0181E00E94700D2091D902F4
:1035C0004091D6055091D7056091D8057091D905E5
:1035D0008091020190910301A0910401B091050135
:1035E000211109C02091E702222339F0480F591F09
:1035F0006A1F7B1F06C02130C9F7481B590B6A0B95
:103600007B0B82E00E94700DC13021F4DF91CF91DD
:103610000C942D11DF91CF910895BF92CF92DF923C
:10362000EF92FF920F931F93CF93DF9300D000D0C0
:10363000CDB7DEB76B017C01042F19821A821B8281
:103640001C820E94111A182F8F3FC1F5C701B601C5
:1036500028EE33E040E050E00E948C3A8091120561
:1036600090E0BC0161507109B12C8B2D90E0861760
:103670009707BCF5FC01EE0FFF1FEE0FFF1FE65191
:10368000FB4FC280D380E12CF12C2C153D054E055B
:103690005F0590F0880F991F880F991FFC01E25178
:1036A000FB4F80819181A0E0B0E0281739074A07DD
:1036B0005B0710F4102F1B0DB394D7CF013061F4CA
:1036C0008091120590E00197212F012E000C330B01
:1036D000281739072CF00EC00F3F39F418162CF4B8
:1036E000100F1F3F41F4013029F0E09112051FEF48
:1036F0001E0F01C010E024E01202C0011124BE011F
:103700006F5F7F4F825D9E4F0E94DD0B89819A81A2
:10371000AB81BC816C017D012DE1F694E794D794D7
:10372000C7942A95D1F7BC01CD019F7169837A8333
:103730008B839C8328EE33E040E050E00E948C3A7B
:1037400084E0189FF0011124E651FB4F60817181E4
:10375000CB01A0E0B0E0281739074A075B0748F023
:1037600082819381A0E0B0E082179307A407B50798
:1037700048F49B01A8EEB3E00E94D33A69837A83B0
:103780008B839C8361E08C2D0E94D00E69817A81AD
:103790008B819C810E94FA170F900F900F900F90D1
:1037A000DF91CF911F910F91FF90EF90DF90CF901D
:1037B000BF900895FF920F931F93CF93DF93EC0177
:1037C000F62E08811981C8010E94323AF81621F0BC
:1037D0006F2DC8010E943A3ACE01DF91CF911F911F
:1037E0000F91FF900895E0915802F09159023FB770
:1037F0004091530250915402F894208190915A02C2
:1038000092239083DA011197F1F798E0608180FFAD
:1038100004C020915B02262B03C020915A0226236C
:103820002083DA011197F1F78695915079F790810D
:1038300080915B02892B80833FBF809153029091DE
:1038400054020197F1F708950F931F93CF93DF93DD
:10385000EC018C01025E1F4F8991882329F00E94A0
:10386000F31BC017D107C1F7DF91CF911F910F91C3
:1038700008951F920F920FB60F9211242F933F932A
:103880004F935F936F937F938F939F93AF93BF9368
:10389000EF93FF932F933F934F935F936F937F9398
:1038A000AF93BF93E0915502F091560290818091C1
:1038B0005702892309F065C0E0914B02F0914C0258
:1038C000908180914A028095892380838091510262
:1038D000909152020197F1F760914F02709150025E
:1038E000A0915502B09156025091570298E080E0A5
:1038F000FB013197F1F7282F30E035952795822F7E
:103900004C91452309F08068915091F79091040300
:10391000911128C0E091DB0491E09E0F9093DB04AD
:103920000E2E000CFF0BE352FC4F8083833749F4CB
:103930008091DA04823094F0973094F090930403ED
:1039400002C094321CF01092DB040AC08F3F41F495
:103950008091DA048F5F8093DA0404C094329CF77C
:103960001092DA0480914D0290914E020197F1F786
:10397000E0914B02F0914C02908180914A02892B98
:103980008083BF91AF917F916F915F914F913F91F4
:103990002F91FF91EF91BF91AF919F918F917F9167
:1039A0006F915F914F913F912F910F900FBE0F90AC
:1039B0001F9018950F931F93CF93DF93D82F07E293
:1039C00015E0C0E0CD1749F0F80161918F0181EE5B
:1039D00095E00E940D03CF5FF5CFDF91CF911F914E
:1039E0000F910895823019F485E395E004C0813089
:1039F00021F488E492E00E94241C8FEF0E94F31BC4
:103A00008FEF0E94F31B8FEF0C94F31BFF920F9329
:103A10001F93CF93DF93F82E95E18902E0011124E3
:103A20008E01075B1A4FC359DD4FB801CE010E94CA
:103A30000C3B892B99F080E38F0D0E941B0CCE016B
:103A40000E94241C81E00E94F21CBE01C801DF918B
:103A5000CF911F910F91FF900C94153BDF91CF9167
:103A60001F910F91FF900895CF92DF92EF92FF92F6
:103A7000CF93DF936A017B0180935301CFE4D1E0C0
:103A800089910E94F31B81E0C935D807C9F784E109
:103A9000E5E3F5E0DF011D928A95E9F72AE0AF0141
:103AA000C701B6010E94D73982E0DF91CF91FF9024
:103AB000EF90DF90CF900C94F21CCF92DF92EF92B8
:103AC000FF92CF93DF936A017B0180935301CFE490
:103AD000D1E089910E94F31B81E0C935D807C9F76D
:103AE00084E1E5E3F5E0DF011D928A95E9F72AE03C
:103AF000AF01C701B6010E94E63982E0DF91CF91A4
:103B0000FF90EF90DF90CF900C94F21CCF93C82FD2
:103B100084E10E941F289C01809124059091250535
:103B2000281739073CF080912205909123058217D0
:103B3000930784F580912005909121052817390776
:103B40003CF080911E0590911F058217930724F584
:103B500080911C0590911D05281739073CF0809134
:103B60001A0590911B0582179307C4F480912201D6
:103B7000811116C0809118059091190528173907F1
:103B80007CF081E0409116055091170542175307CC
:103B900044F406C082E005C081E003C083E001C0B8
:103BA00080E0C13029F490912101982B909321015C
:103BB000CF9108950F931F9386E00E94480460E020
:103BC00082E00E94A4250E94762820911D014AE0EF
:103BD000249F900111248901330F220B330BDC0148
:103BE000CB01800F911FA21FB31F8093E30290931C
:103BF000E402A093E502B093E6021F910F910895AD
:103C00000F931F9380910201909103010E940F2650
:103C100061E082E00E94A4250E94762820911D0187
:103C20004AE0249F900111248901330F220B330BAA
:103C3000DC01CB01800F911FA21FB31F8093E30211
:103C40009093E402A093E502B093E6021F910F91D6
:103C500008950F931F93CF93C0910803C23009F0CA
:103C600085C00E942B242091E002892B69F5213028
:103C700099F40E947628DC01CB0188539F4FAF4F07
:103C8000BF4F8093310590933205A0933305B093D5
:103C90003405C093E0026AC0223009F053C00E948C
:103CA000762800913105109132052091330530912D
:103CB0003405061717072807390708F043C081E0C5
:103CC0008093DE0283E03BC02230A1F50E9476287B
:103CD0000091310510913205209133053091340562
:103CE000601771078207930748F58091DF02282F3C
:103CF00030E09091E102882341F0833070F4F901C3
:103D0000E652FD4F4081491741F08F5F8093DF02FB
:103D1000F901E552FD4F908309C0F901E652FD4FCC
:103D2000208129130BC081508093DF0281E08093B2
:103D3000DA0204C0233011F41092DE0281E0809395
:103D4000E00214C08091E002833081F40E94762862
:103D5000DC01CB0188539F4FAF4FBF4F809331059C
:103D600090933205A0933305B0933405CF911F9102
:103D70000F910895AF92BF92CF92DF92EF92FF9290
:103D80000F931F93CF93DF93CDB7DEB727970FB66F
:103D9000F894DEBF0FBECDBFE82F8E3321F08C33F9
:103DA00009F040C009C0E0905F02EE2009F40CC1A8
:103DB000F12C00E010E00FC08FEF93E00E942D0C7B
:103DC00090E0009709F400C101EF10E0081B190B07
:103DD00071EFE72EF12CE016F10608F4F5C0C801EA
:103DE000825F9C4F0E942D0C0E94BA1E0E94291EC9
:103DF0008091DA02813021F41092DA020E942D11B2
:103E00000E151F0560F480911F01909120019C0107
:103E1000220F331F64E0820F931F0E9493190F5FDC
:103E20001F4FD9CF8FEB8E0F8A31D8F40E2E000C96
:103E3000FF0BE758FC4FE4911E2F12951F70DE0117
:103E4000119680E090E0F0E0811708F08CC09F01AF
:103E5000082E01C0220F0A94EAF728702D930196CC
:103E6000F3CF80ED8E0F8A30B8F4DE01119620E09A
:103E700030E00E2E000CFF0BE159FC4F8491022E16
:103E800001C0880F0A94EAF780718D932F5F3F4F2E
:103E90002530310599F764C0E032D9F480911F01D3
:103EA0009091200164E0880F991F880F991F279631
:103EB0000FB6F894DEBF0FBECDBFDF91CF911F913B
:103EC0000F91FF90EF90DF90CF90BF90AF900C9448
:103ED0009319E43299F4FE01319680E090E042E1DA
:103EE00050E09A01082E01C0220F0A94EAF72078C8
:103EF0002193019687309105A1F734C020E030E08E
:103F00008E2FEE0F990BF901E757FC4FE491F0E08B
:103F1000E817F907F9F4F901ED58FC4FE4911E2F69
:103F200012951695169513701D5FAE014F5F5F4F8A
:103F3000DA0182E090E0F0E09F01082E01C0220F3C
:103F40000A94EAF720782D9301962A2F241B211733
:103F500098F309C02F5F3F4F26313105A1F634C0D9
:103F600015E001C017E0CE0101965C01E12CF12CB7
:103F7000C12ED12C91E0C91AD108E11628F50E9472
:103F8000001EF50121915F0180911F019091200198
:103F9000211102C064E006C09C01220F331F64E0BF
:103FA000820F931F0E9493190E94DA1DCE14DF0422
:103FB00039F064E080911F01909120010E949319D3
:103FC000FFEFEF1AFF0AD9CF27960FB6F894DEBF9E
:103FD0000FBECDBFDF91CF911F910F91FF90EF905A
:103FE000DF90CF90BF90AF9008952F923F924F9265
:103FF0005F926F927F928F929F92AF92BF92CF9279
:10400000DF92EF92FF920F931F93CF93DF93C82F0E
:1040100081EE95E00E94D502892B19F410923005AB
:10402000B9C381EE95E00E94D50205970CF046C019
:10403000C0913005CC2359F10E94762800912C05BF
:1040400010912D0520912E0530912F050617170789
:104050002807390790F4C0E081EE95E00E94D50270
:104060002C2F30E028173907CCF681EE95E00E941E
:10407000B30280933005CF5FEFCF81EE95E00E94D1
:10408000D5022C2F30E0281739070CF083C381EEBE
:1040900095E00E94D502809330050E947628DC01CD
:1040A000CB018C509E4FAF4FBF4F80932C05909308
:1040B0002D05A0932E05B0932F056CC307E215E0E4
:1040C000BCE2CB2EB5E0DB2E780181EE95E00E94BC
:1040D000B302D7018D937D01CA16DB06B1F780913B
:1040E0002605813009F456C321E0209326059091DE
:1040F0002B05983809F4FFC0C0F4973009F4D8C0F4
:1041000050F4923009F482C0933009F485C09130A4
:1041100009F032C324C0913809F4F8C0923809F488
:1041200078C0983009F028C3E6C09C3D09F4F2C17C
:1041300050F49C3B09F41AC29B3D09F4EFC09B3B31
:1041400009F01AC33FC19E3D09F4C9C208F4B7C2C1
:10415000973E09F4E2C2973F09F4ECC20DC3C25086
:10416000C23018F40E944C0B0BC3EBE2F5E020E0E8
:1041700030E0A901AAE0B0E00E94E23AD801CD9176
:104180008D014C2F50E09A01A4E035952795AA9512
:10419000E1F76901330FEE08FF08A7019601260F2A
:1041A000371F481F591FAAE0B0E00E94E23ACF70C3
:1041B0009B01AC012C0F311D411D511DE017F10772
:1041C000C9F6809106038111D7C20E94E23A00919C
:1041D000D6051091D7052091D8053091D9056017E3
:1041E00071078207930709F4C7C28B019C01085B22
:1041F0001B402109310909341B472349334008F08A
:10420000BBC20E94FA170E942D11B6C22093DC0394
:10421000B3C21092DC03B0C26091D6057091D7058D
:104220008091D8059091D9052AE030E040E050E037
:104230000E948C3A69017A01CBE2D5E06AE0862ED1
:10424000912CA12CB12C74E6472E512C612C712C91
:10425000C701B601A50194010E948C3A262ECA011D
:10426000B901A50194010E948C3A362E329450EF88
:1042700035223228C701B601A30192010E948C3A6F
:1042800069017A013A920C171D0711F78091D90242
:10429000811109C08091E702882311F081E004C0F8
:1042A00010922B0503C082E080932B0585E04DC260
:1042B000C250C23018F40E944C0B62C280910603B7
:1042C00081115AC280912705823019F42093D902B6
:1042D00009C01092D902813019F48093E70202C01C
:1042E0001092E7026091D6057091D7058091D805AC
:1042F0009091D90586CF80910603811144C2C250A6
:10430000C23008F025C20E944C0B3AC2C250C230E3
:1043100010F00E94F90E0E944C0B32C2009127054A
:1043200010912805E12EF12CFE2CEE24E00EF11C5C
:10433000C0912A05D0E0DC2FCC2780912905C80F39
:10434000D11D82E090E00E944F24063101F5183E15
:10435000F1F4C1E0D1E0D093A305C093C50510925C
:10436000A4051092C60581E00E942225811106C095
:104370006C2F81EE95E00E940D0304C080E090E078
:104380000E944F24CF5FCF3731F712E015C0C12C08
:10439000D12C12E0CC15DD0579F0C7018C0D9D1DE7
:1043A0000E942D0C180F682F81EE95E00E940D03DE
:1043B000EFEFCE1ADE0AEECF612F81EE95E00E947C
:1043C0000D03DAC1909127058091280510922705E9
:1043D00010922805803609F462C0C8F4873509F4C4
:1043E0004BC040F48734C1F18535F1F1853409F0D3
:1043F0008FC02DC08E3509F444C008F04BC08C35F9
:1044000009F086C082EB8093270582E47FC087365F
:1044100009F458C060F4823609F447C0C0F183360D
:1044200009F076C082EB8093270585EA6FC0883754
:1044300009F44CC020F4893609F448C069C08A37B1
:1044400009F45AC0833B09F063C08DE45FC0933028
:1044500009F05EC080ED5AC0933009F059C08CED70
:104460008093270580EE52C080916201843111F45F
:1044700081E849C080E847C080EC8093270580E44C
:1044800045C0809115058093270585E23FC0809146
:10449000140501C082E38093270588E037C080912E
:1044A0001D018093270582E331C060911F01709147
:1044B000200180EB94E00E94643A645060932705E9
:1044C00082EB24C082EB8093270520C08091D90223
:1044D000811106C08091E702882341F081E004C089
:1044E0008150823018F482E080932705809127055F
:1044F000882371F080E207C08091DC03882311F0EB
:104500008FEF01C08FE78093270502C080932805B5
:1045100082E01BC170912805609129052091270533
:10452000872F90E0820F911D40912A0550E09C0159
:10453000260F311D33274217530719F086E590E007
:1045400012C0FFEF7F9F800D911D11248B3423E358
:10455000920729F4613529F40C94000002C00E94EE
:104560002B0C87E790E00E944F2406C1809128051C
:104570001092270510922805C250C23008F4ABC033
:10458000803609F484C028F4853519F18E3581F11F
:10459000A2C0813609F44FC0823609F09CC06091F8
:1045A00029056F7370E06C5F7F4F80EB94E00E9491
:1045B000783A7093200160931F0165ED73E080E00D
:1045C0000E9490126FE171E08CE190E00E94980BE4
:1045D0006DC0909129058091620190FF06C08431E1
:1045E00009F479C00E94F90E76C08031D9F773C002
:1045F000809129058F7080931505209114058111F4
:1046000003C0222309F467C032E3839FC001112451
:10461000845D9E4F820F911D092E000CAA0BBB0BCF
:104620008093020190930301A0930401B0930501CC
:1046300063E074E022C0209129052F7720931405B0
:1046400080911505811103C0222309F444C042E37F
:10465000849FC0011124845D9E4F820F911D092EFD
:10466000000CAA0BBB0B8093020190930301A09353
:104670000401B093050161EF73E080E00E949012A5
:1046800062E071E088E190E00E94650B0FC08091CC
:10469000290580931D0163EE73E080E00E94901273
:1046A0006DE171E082E091E00E94030C6CE271E048
:1046B00080E090E00E943C280E948C120CC0E091A7
:1046C0002705F0E0EC59FE4F80810E941F2890934F
:1046D00027058093280582E00E94DA1C4DC0809156
:1046E000270580939A028091290590E0982F8827CA
:1046F00020912805820F911D909399028093980232
:104700006091D6057091D7058091D8059091D90513
:104710000E94FA170E94250E2FC0E091FD02E15081
:10472000E83028F4F0E0E857FE4F808101C080E0D7
:104730008F7008C080910603811102C080E801C01B
:1047400080E0885F8093270581E00E94DA1C18C012
:10475000983091F481E08093070361E080E00E944B
:104760003F1A80910803882339F01092080365E10D
:1047700074E080E00E94901280E090E00E944F245C
:104780001092260507C09830B9F30E94391910928B
:104790000703F2CFDF91CF911F910F91FF90EF9020
:1047A000DF90CF90BF90AF909F908F907F906F9051
:1047B0005F904F903F902F900895833081F028F4C0
:1047C000813099F08230A1F008958730A9F08830C7
:1047D000B9F08430D1F4809180008F7D03C0809146
:1047E00080008F7780938000089584B58F7702C012
:1047F00084B58F7D84BD08958091B0008F7703C00C
:104800008091B0008F7D8093B00008953FB7F894F9
:104810008091770590917805A0917905B0917A05FE
:1048200026B5A89B05C02F3F19F00196A11DB11D0B
:104830003FBFBA2FA92F982F8827820F911DA11D46
:10484000B11DBC01CD0142E0660F771F881F991F83
:104850004A95D1F70895CF93DF93EAE9F4E0849184
:10486000E6E8F4E0D491E2E7F4E0C491CC2391F0DF
:1048700081110E94DD23EC2FF0E0EE0FFF1FE95ABB
:10488000FB4FA591B491EC91ED2381E090E021F4F0
:1048900080E002C080E090E0DF91CF910895682F22
:1048A00081EE95E00C940D03CF92DF92EF92FF9290
:1048B00080916201C090D605D090D705E090D805D0
:1048C000F090D905803109F041C0C0925A01D092D0
:1048D0005B01E0925C01F0925D010E944D0F8093BC
:1048E000D4058091D0059091D105A091D205B091C9
:1048F000D305C816D906EA06FB06B1F06AE571E0F1
:1049000080E190E00E94650B80915A0190915B01DB
:10491000A0915C01B0915D018093D0059093D10589
:10492000A093D205B093D3059091D4058091CF0583
:10493000981709F44AC064ED75E080E091E00E94A8
:10494000030C8091D4058093CF053FC0C0925E01D7
:10495000D0925F01E0926001F09261010E944D0FE0
:104960008093D5058091CB059091CC05A091CD0584
:10497000B091CE05C816D906EA06FB06B1F06EE581
:1049800071E084E190E00E94650B80915E0190915E
:104990005F01A0916001B09161018093CB0590937C
:1049A000CC05A093CD05B093CE059091D50580910F
:1049B000CA05981751F065ED75E081E091E00E941D
:1049C000030C8091D5058093CA05FF90EF90DF908E
:1049D000CF9008952091C905892B51F420FD03C083
:1049E00060E374E002C065E474E080E00C9490122F
:1049F00020FD06C021602093C9056EE374E005C068
:104A00002E7F2093C90568E374E080E00E94901235
:104A10001092C8050895209162019091C7058130D8
:104A200039F4203111F082E001C081E0892B06C009
:104A3000203111F08DEF01C08EEF89238093C705DF
:104A40000C946511282F3091C605313208F04AC008
:104A50008091A2058111FCCF9091C50542E0409361
:104A6000A2052093A1052FEF2093A00510929F058A
:104A700030939E05E5EAF5E0AEE7B5E020E03217B9
:104A800021F041914D932F5FFACF10927D05209137
:104A90007D05990F922B90937D0590917C05913027
:104AA00061F410927C0590917D059093BB009091EC
:104AB000BC0093FDF8CF95EC01C095EE9093BC003F
:104AC0009091A2059230E1F39091A0059F3F79F07B
:104AD0008091A005803241F08091A005803331F0B3
:104AE00084E005C081E003C082E001C083E0109251
:104AF000A4051092C6051092A30508950F931F9365
:104B0000CF93DF938B0190917B0521E02093A30548
:104B10009093C5051092A4051092C605682F8EE7E4
:104B200096E00E941304E80119E0115031F06991F8
:104B30008EE796E00E941304F8CF81E0DF91CF91D9
:104B40001F910F910C9422251F93CF93DF93282F51
:104B500030E0F901E757FB4F8491F901EB58FB4F27
:104B6000D491F901EF59FB4FC491CC23C1F0162F1A
:104B700081110E94DD23EC2FF0E0EE0FFF1FE45BBC
:104B8000FB4FA591B4919FB7F894111104C08C917B
:104B9000D095D82302C0EC91DE2BDC939FBFDF9130
:104BA000CF911F910895CF93DF9390E0FC01EB58D4
:104BB000FB4F2491FC01EF59FB4F8491882361F155
:104BC00090E0880F991FFC01EA5DFB4FC591D491DD
:104BD000FC01E45BFB4FA591B491611109C09FB743
:104BE000F8948881209582238883EC912E230BC032
:104BF000623061F49FB7F8948881322F3095832317
:104C00008883EC912E2B2C939FBF06C08FB7F8940E
:104C1000E8812E2B28838FBFDF91CF9108958F924B
:104C20009F92AF92BF92CF92DF92EF92FF921F932B
:104C3000CF93DF93EC0180916301863021F08F3FA9
:104C400009F0F1C104C0E6E5F4E014916FC086E01C
:104C500080936301E6E5F4E014911F3F09F4E3C19A
:104C6000113009F440C030F1123009F05FC01092E9
:104C7000B0001092B1008091B00082608093B000CB
:104C80008091B10081608093B100E7E6F4E0E491A7
:104C9000F0E0EE0FFF1FE45BFB4F85919491909342
:104CA000DC058093DB05EBE7F4E0E491E093DA05C3
:104CB00012E0B4C114BC15BC84B5826084BD85B556
:104CC000816085BDE7E6F4E0E491F0E0EE0FFF1FC0
:104CD000E45BFB4F85919491EBE7F4E0E491E09382
:104CE0008B0610E09BC11092800010928100809191
:104CF0008100886080938100809181008160809331
:104D00008100E7E6F4E0E491F0E0EE0FFF1FE45BE2
:104D1000FB4F85919491EBE7F4E0E491E0938A06F0
:104D200061E086E00E94D32511E0A5C017FD7BC19C
:104D300061E086E00E94D325812F8D7F09F09BC022
:104D40006E01E12CF12C60E072E18AE790E0A701AE
:104D500096010E94AE3A49015A01BA01A901415097
:104D60005109610971094F3F51056105710509F04C
:104D700008F445C060E472E48FE090E0A70196017A
:104D80000E94AE3ABA01A901415051096109710965
:104D90001230E9F44F3F51056105710509F008F43F
:104DA000DDC060E970ED83E090E0A70196010E940C
:104DB000AE3ABA01A90141505109610971094F3F49
:104DC00051056105710509F020F583E04DC04F3FA5
:104DD000510561057105A9F0A0F068E478EE81E065
:104DE00090E0A70196010E94AE3ABA01A901415094
:104DF000510961097109112309F4E1C0D8C081E0AA
:104E000001C082E0111130C095B5987F892B85BD16
:104E100069C068E478EE81E090E0A70196010E9405
:104E2000AE3ABA01A90141505109610971094F3FD8
:104E300051056105710509F008F48EC064E274EF54
:104E400080E090E0A70196010E94AE3ABA01A90164
:104E500041505109610971094F3F510561057105C3
:104E600011F008F07DC085E09091B100987F892B0A
:104E70008093B10031C06E01E12CF12C60E072E151
:104E80008AE790E0A70196010E94AE3ABA01A90113
:104E900041505109610971094115510581E06807C7
:104EA000710580F068E478EE81E090E0A70196015A
:104EB0000E94AE3ABA01A901415051096109710934
:104EC00083E001C081E0113039F490918100987F36
:104ED000892B8093810018C01130B1F0123049F154
:104EE0001111A1C047BD8FEF9FEFDC0180939006A9
:104EF00090939106A0939206B093930680916E00D2
:104F0000826080936E008FC0509389004093880028
:104F10008FEF9FEFDC0180938C0690938D06A0931A
:104F20008E06B0938F0680916F00826080936F0031
:104F30007AC04093B3008FEF9FEFDC018093DD05D3
:104F40009093DE05A093DF05B093E005809170009B
:104F500082608093700067C084E086CF82E084CF57
:104F600062E17AE780E090E0A70196010E94AE3A04
:104F7000BA01A90141505109610971094F3F510519
:104F80006105710591F088F0D501C4012AE0B5955D
:104F9000A795979587952A95D1F7AC01BD0141500A
:104FA00051096109710987E05FCF86E05DCF4F3F0E
:104FB00051056105710509F098F684E023CF4F3F54
:104FC00051056105710541F138F162E17AE780E050
:104FD00090E0A70196010E94AE3ABA01A9014150A2
:104FE0005109610971094F3F51056105710591F042
:104FF00088F0D501C4013AE0B595A79597958795B6
:105000003A95D1F7AC01BD014150510961097109CF
:1050100085E0FACE84E0F8CE83E0F6CE61E086E06B
:105020000E94D3258DCEDF91CF911F91FF90EF90FD
:10503000DF90CF90BF90AF909F908F9008958E306B
:1050400008F08E502091590190E4299F900111247D
:105050008770822B80937C0080917A00806480939B
:105060007A0080917A0086FDFCCF809178002091B3
:10507000790090E0922B08958F929F92AF92BF9209
:10508000CF92DF92EF92FF926B017C010E94062487
:105090004B015C01C114D104E104F104F1F00E9460
:1050A0000624DC01CB0188199909AA09BB09883EAD
:1050B0009340A105B10570F321E0C21AD108E108BF
:1050C000F10888EE880E83E0981EA11CB11CC11463
:1050D000D104E104F10419F7DDCFFF90EF90DF90E8
:1050E000CF90BF90AF909F908F9008952FB7F89476
:1050F00060917305709174058091750590917605A6
:105100002FBF08951F920F920FB60F9211242F9365
:105110003F938F939F93AF93BF938091730590912B
:105120007405A0917505B09176053091940623E041
:10513000230F2D3720F40196A11DB11D05C026E8CF
:10514000230F0296A11DB11D209394068093730531
:1051500090937405A0937505B093760580917705BB
:1051600090917805A0917905B0917A050196A11DDD
:10517000B11D8093770590937805A0937905B0933E
:105180007A05BF91AF919F918F913F912F910F9091
:105190000FBE0F901F901895CF93DF93CDB7DEB75A
:1051A00029970FB6F894DEBF0FBECDBF789484B5B3
:1051B000826084BD84B5816084BD85B5826085BD13
:1051C00085B5816085BD80916E00816080936E00A1
:1051D0001092810080918100826080938100809193
:1051E0008100816080938100809180008160809344
:1051F00080008091B10084608093B1008091B00004
:1052000081608093B00080917A00846080937A00FE
:1052100080917A00826080937A0080917A00816028
:1052200080937A0080917A00806880937A0010924F
:10523000C10061E089E00E94A42561E089E00E944C
:10524000D325EEE7F4E0849180935B02E491E0954E
:10525000E0935A02EAE6F4E0E491F0E0EE0FFF1F7B
:10526000E45BFB4F8591949190935902809358028F
:1052700060E088E00E94D32561E088E00E94A425D8
:10528000EDE7F4E0E491E0935702E9E6F4E0E4911D
:10529000F0E0EE0FFF1FE95AFB4F85919491909338
:1052A0005602809355028DE991E0909354028093C9
:1052B00053028DEB90E090935202809351028BE960
:1052C00091E09093500280934F028CE291E0909392
:1052D0004E0280934D028091680081608093680047
:1052E0008BE690E090934C0280934B0211E0109378
:1052F0004A0280915302909154020197F1F78091F4
:105300006B00816080936B0044E150E060E270E0EC
:105310008DE692E00E94FA3A44E150E060E270E0EB
:1053200082E892E00E94FA3A10929702E091F10529
:10533000F091F20582E08083E091ED05F091EE05B9
:105340001082E091EF05F091F00583E380831092E5
:10535000F905E091F505F091F60586E08083E0918E
:10536000F305F091F405808180618083E091F3057D
:10537000F091F405808188608083E091F305F091DD
:10538000F405808180688083E091F305F091F40555
:1053900080818F7D808381EE95E00E945A030E9478
:1053A00010131093590162E08EE00E94D32562E051
:1053B0008FE00E94D32562E080E10E94D32562E065
:1053C00081E10E94D32562E084E10E94D32560E060
:1053D00085E10E94D32561E086E00E94D32560E04C
:1053E00086E00E94A42561E087E00E94D32560E06A
:1053F00087E00E94A42561E085E00E94D32561E05A
:1054000084E00E94D32561E083E00E94D32560E020
:1054100085E00E94A42560E084E00E94A42560E06D
:1054200083E00E94A42561E082E00E94D32560E031
:1054300082E00E94A42580915F028F7780935F02B3
:1054400060E08091D4050E94D00E0E94640E6091AD
:105450005A0170915B0180915C0190915D016093B4
:10546000D6057093D7058093D8059093D90560939E
:1054700000037093010380930203909303030E943F
:10548000FA1762E084EF91E00E9493194091E802DC
:105490005091E9026091EA027091EB0281E30E946F
:1054A000341D4091EC025091ED026091EE0270913A
:1054B000EF0282E30E94341D4091F0025091F1020C
:1054C0006091F2027091F30283E30E94341D4091D7
:1054D000F4025091F5026091F6027091F70284E3B4
:1054E0000E94341D4091F8025091F9026091FA0235
:1054F0007091FB0285E30E94341D6091010188E6F2
:105500000E945F0F40915D0250915E02052E000CDB
:10551000660B770B88E60E94341D40915C0250E0D8
:1055200060E070E08FE60E94341D4091FF0250E081
:1055300060E070E080E70E94341DBE016F5F7F4F26
:1055400082E093E00E94DD0B49815A816B817C816E
:1055500081E70E945D1D86E70E941B0C84EB91E0B1
:105560000E94241C81E00E94F21CE0905F02F12C5A
:1055700083E60E941B0C00E010E00E151F0554F49A
:10558000C801825F9C4F0E942D0C0E94F31B0F5F8D
:105590001F4FF3CF81E00E94F21C61E08DE60E9474
:1055A0005F0F1092000160E080E30E945F0F0E9495
:1055B0002D11E0900803E11050C78091070381117D
:1055C00020C08091E3029091E402A091E502B091A5
:1055D000E602892B8A2B8B2BA1F40E942B24892B8A
:1055E00031F480910603882311F40C9450360E9404
:1055F0002B24019731F480910603813011F40C942F
:105600005C360E94150D019611F40C948F3362E301
:1056100070E080E090E00E943C280E94150D2C0173
:105620008F3F4FEF940711F40C948F338837910517
:1056300009F073C681E00E94720F1092B7030E94B6
:10564000490D892B29F160E082E390E00E949319D3
:105650009091B70381E0890F8093B703943131F4BF
:1056600063EE72E080E00E949012E9CF893238F355
:10567000909162018091C705903119F480958170F5
:1056800004C08695817091E089270E940B253EC653
:1056900062E370E080E090E00E943C288091B703D4
:1056A000853108F46AC066ED72E081E00E949012D4
:1056B000FF24F39400E010E00E94490D892B09F0CB
:1056C0004EC060E082E390E00E949319FF20F9F061
:1056D0006CEB71E08AEB92E00E94153BE091FC02DA
:1056E00064E0E69FF0011124EC51FD4F4AE06CE9C3
:1056F00072E0808191810E94CC396CE972E08AEB82
:1057000092E00E94013B8AEB92E00E946C110E94A1
:10571000920C009711F4F12CCFCF181619061CF437
:1057200081E090E002C08FEF9FEF080F191F009FEC
:10573000C001019F900D900D1124499764F3809151
:10574000FC0217FF05C0823008F4B2CF815004C0BC
:10575000853008F0ADCF8F5F8093FC02A9CF6CEF4E
:1057600072E086E591E00E94030C60E084EF91E036
:105770000E9493190E946511C9C582E08093C805F3
:1057800010929B02212C312C8091C805882309F4AA
:10579000BDC50E94920C8C010E94490D9C011016FF
:1057A000110674F48091B603020D131D882321F0B5
:1057B000003F11058CF011C0063911056CF00DC0C9
:1057C0000115110551F0C101801B910B863F9F4FC0
:1057D00024F0200E311E01C01801C1016AE070E002
:1057E0000E94783A6731710508F0B3C3FB01EC5CA5
:1057F000FF4F0C94CD3A232B19F469EC72E0C2C030
:1058000002E016E10E94490D892BF9F060E082E385
:1058100090E00E9493191150A9F78091D802882333
:1058200029F01092D80261EC72E004C00093D80213
:1058300068EB72E080E00E94901260E088EE93E0F6
:105840000E9493190E946511DCCF67EA72E080E044
:105850000E9490128091D8029EEF980F923018F01B
:1058600086568230C8F4C090D605D090D705E09017
:10587000D805F090D905C701B6010E94111A082F6A
:1058800087FD0AC00E944D0F282F30E040E050E015
:10589000C701B6010E94D9190E94261900E010E044
:1058A0000E94490D892B09F05FC00E94920C9C0157
:1058B000892B09F453C09091D8028EEF890F823062
:1058C00008F43FC096569230E0F18091D605909151
:1058D000D705A091D805B091D90537FF0EC0813CFE
:1058E000E6EC9E07EDE2AE07B105B8F0BC01CD01D4
:1058F00060547D40834091090EC0803843EC94078A
:1059000049ECA40741E0B40740F4BC01CD01605C60
:10591000724F8C4F9F4F0E94FA178091D60590913D
:10592000D705A091D805B091D90581389649A849E5
:10593000B10520F081E08093E7020EC01092E702EB
:105940000BC037FF02C00C9460360430110514F010
:105950000C946F360F5F1F4F0E942D1160E084E1A1
:1059600090E00E9493199CCF0E94542460E084EF41
:1059700091E0CCC2232B69F480916201803131F433
:1059800069E972E080E00E949012BCC46BE872E0AA
:10599000F9CF0E94F90EB6C4232B19F46EE772E01A
:1059A000F1CF8091D90281110AC08091E70288234A
:1059B00061F0813069F4AA24A394B12C0CC0813029
:1059C00039F452E0A52EB12C06C0A12CB12C03C095
:1059D00043E0A42EB12C24E0C22ED12C37ECE32ED0
:1059E00031E0F32E01E010E023E030E040E050E051
:1059F000B5018BE090E00E94AA11A816B906E1F06B
:105A0000009729F41092D9021092E70213C0813056
:105A1000910531F41092D90281E08093E7020AC027
:105A20008230910511F481E003C0039719F482E0FC
:105A30008093D9020E9454240E94250E0C9497361C
:105A4000C9010E94B7125EC4232B51F480919A02BF
:105A5000813019F46DE672E095CF60E672E092CF86
:105A600081E080939A02609198027091990282E09D
:105A7000C82ED12C98EDE92E91E0F92E02E310E02A
:105A800020E23EE440EE51EB82E090E00E94AA1159
:105A9000909399028093980260E084EF91E00E94D5
:105AA00093190E94490D892B11F00C948136809135
:105AB000980290919902892B11F40C94813668E92F
:105AC00072E08BE691E00E94980B0C94B4366091E2
:105AD0009702232B41F4662319F064E572E052CF5C
:105AE0006CE472E04FCF70E012E0C12ED12C0CEDCF
:105AF000E02E01E0F02E05E010E02AEF30E040E07B
:105B000050E085E090E00E94AA118093970260E047
:105B100084EF91E00E9493190E94490D892B11F0A6
:105B20000C94953680919702882311F40C94953645
:105B30000C94B43660911F017091200180EB94E0C9
:105B40000E94643A5B01232BE9F460EE71E08AEB7A
:105B500092E00E94153B4AE06CE972E0C5010E94A8
:105B6000CC396CE972E08AEB92E00E94013B64EE72
:105B700071E08AEB92E00E94013B8AEB92E00E9486
:105B80006C11C0C3A3E0CA2ED12CB0EFEB2EB1E054
:105B9000FB2E01E010E022E330E043E050E080E043
:105BA00090E00E94AA11BC0180EB94E00E94783A38
:105BB0007093200160931F016FE171E08CE190E030
:105BC0000E94980B0C94B436C9010E94EA129AC341
:105BD000232B19F46CE272E0D5CE80E006C0232BB3
:105BE00019F46CE372E0CECE81E00E94CE098AC344
:105BF000232B19F46FE172E0C5CE64EC73E081E20F
:105C000093E00E94D30B80E293E00E942D0C833737
:105C100099F48091C403882379F00C94A236232B45
:105C200019F461E072E0AECE8BEB91E00E942D0C96
:105C30008093B503811103C00E94E01263C31982EF
:105C40001A821B821C821E821D8260E084EF91E01A
:105C50000E94931999249A942FEF2987712C10E0B0
:105C6000FAE06F2E0E94920C112321F097FF02C0E0
:105C7000115014C0181619068CF4212F30E0711041
:105C800085C08091B5034AE0849FC001112402972A
:105C90008217930714F40C948C391F5F812F662DA3
:105CA0000E94583A082F71107AC05985501709F48C
:105CB00060C06EE20602700111246DE072E080E0C7
:105CC0000E949012BE2C64E0A62EAE0C73E7C72E85
:105CD00072E0D72EEEE08E2E8E0CAB1468F08B1493
:105CE00059F08B2D90E084549E4F0E942D0CD601CC
:105CF0008D936D01B394F1CF80E00E94061D570192
:105D0000BFE3AB1ABEEFBB0A51E1C52E53E0D52E5F
:105D1000E6E1EE1AEEEFFE0AC5010E942D0C982F67
:105D20009370D6019C93282F30E0A9015595479593
:105D300055954795437011964C93119744E03595CE
:105D400027954A95E1F7237012962C931297829526
:105D500086958695837013968C93BFEFAB1ABB0A1A
:105D6000E4E0CE0ED11CAE14BF04B1F60987712C4D
:105D700079CF0E94490D892BD1F360E084EF91E047
:105D80000E9493197724739410E06CCF2D31310564
:105D90000CF483CF812F662D0E94583A082FF1E032
:105DA0007F1260CF901609F457C02EE00202600106
:105DB0001124BE016F5F7F4FC6018F569E4F0E9418
:105DC000DD0BBE016B5F7F4FC6018B569E4F0E945D
:105DD000BF0B560149E6A41A4EEFB40AB6E18B2E6A
:105DE000B1E09B2E760154E6E51A5EEFF50AC50197
:105DF0000E942D0CD4018D934D01BFEFAB1ABB0A4D
:105E0000EA14FB04A1F7ADE0AA2EA1E0BA2EE1E668
:105E1000CE1AEEEFDE0AC7010E942D0CD5018D933C
:105E20005D01BFEFEB1AFB0ACE14DF04A1F720914E
:105E300018012F708091190190911A0198278927D4
:105E40009827A0E0B0E0A22B80930D0390930E035F
:105E5000A0930F03B09310030E942B24892B19F4F5
:105E600064EF71E002C06BEF71E08CE992E00E9498
:105E7000153B69817A818B819C81ECE9EE2EE2E011
:105E8000FE2EFFE0CF2ED12C611571058105910505
:105E9000A1F096012B7F2830310511F42EE20EC0BF
:105EA0002AE030E040E050E00E948C3A605DD7018B
:105EB0001F966C93B901CA0103C020E2F70127873E
:105EC00041E0C41AD10851E0E51AF108A5E0CA166C
:105ED000D104D1F66CE972E081E00E943111809129
:105EE000040381110E9487060E942B24892B09F448
:105EF00041C780919B02813009F43CC70E94490D43
:105F0000892B09F434C760E088EE93E00E9493196E
:105F100034C1232B51F48091FE02811103C064EF40
:105F200071E031CD66EE71E02DCD0E945506EAC1DB
:105F30009091B603232B41F4911103C061ED71E000
:105F400021CD6BED71E01ECD81E089278093B603F2
:105F50000BC7232B09F011C166EC71E013CD232B85
:105F600019F465EB71E00ECD63EA71E081E00E9407
:105F7000901261E971E080E00E94901260E088EE8A
:105F800093E00E949319C0906902D0906A02E09059
:105F90006B02F0906C021092690210926A021092E9
:105FA0006B0210926C0280EC90E7A7E2B4E380935E
:105FB000060190930701A0930801B0930901409155
:105FC000650250916602609167027091680280E0FC
:105FD0000E94700D6091D6057091D7058091D8050B
:105FE0009091D9050E94FA1762E072E08AEB92E084
:105FF0000E94153B6091690270916A0280916B0268
:1060000090916C022EE232E240E050E00E94AE3A03
:10601000CA01B9012AE04CE952E00E94D7396CE983
:1060200072E08AEB92E00E94013B8AEB92E00E94D0
:106030006C110E942B24019709F079C00E94490D30
:10604000892B09F41DC773C0232B19F464E671E092
:1060500099CCC0906502D0906602E0906702F09003
:10606000680260E571E081E00E9490126FE371E0E8
:1060700081E00E94901260E088EE93E00E94931904
:1060800040916502509166026091670270916802CA
:1060900080E00E94700D60916502709166028091AF
:1060A0006702909168020E9470110E942B24019750
:1060B00009F09DC70E94490D892B09F452C797C763
:1060C000232B19F464E271E05DCCC0906102D090A2
:1060D0006202E0906302F090640263E171E081E0AB
:1060E0000E94901260E088EE93E00E949319409124
:1060F000610250916202609163027091640280E0DB
:106100000E94700D60916102709162028091630241
:10611000909164020E9470110E942B24019709F053
:106120007DC70E94490D892B09F4AEC777C70E942D
:106130002B24892B09F09BC660E871E081E00E9466
:10614000901260E771E080E00E94901269E672E0D0
:1061500080E090E00E94650B60E080ED97E00E9497
:1061600093190E94640E6091D6057091D7058091B5
:10617000D8059091D9050E94FA170E946511F4C5BF
:10618000232B19F469EE70E0FDCB60910201709150
:10619000030142E0C42ED12C57E0E52E52E0F52E4B
:1061A0000AE010E020ED37E044E650E081E090E0C6
:1061B0000E94AA11092E000CAA0BBB0B80930201AE
:1061C00090930301A0930401B093050186E00E941F
:1061D000480468EF70E080E00E94901262E071E095
:1061E00088E190E00E94650BBFC560911D019AE0B7
:1061F000699FB0011124232B19F469ED70E0C2CB23
:1062000022E0C22ED12C3CE0E32E32E0F32E0AE055
:1062100010E024EC39E043E050E080E090E00E94A0
:10622000AA116AE070E00E94783A60931D016DE166
:1062300071E082E091E025C060911E0170E0660F80
:10624000771F232B19F46AEC70E09CCB02E0C02E80
:10625000D12C8CE0E82E82E0F82E02E010E024EF52
:1062600031E040E050E080E090E00E94AA1197FD0C
:1062700001969595879580931E016EE171E083E00C
:1062800091E00E94030C70C5232B19F468EA70E0BA
:1062900079CB6091600270E0A5E0CA2ED12CB2E10A
:1062A000EB2EB2E0FB2E01E010E022E030E040E017
:1062B00050E08BE090E00E94AA11182F69EB70E08B
:1062C00080E00E9490121093600260E672E086E621
:1062D00091E00E94030C90916002911103C0109212
:1062E000220142C581E080932201809121019130F9
:1062F00011F48F7E01C080618093210135C5C901F1
:106300000E94EA2480E00E94F51F3ECA80910803A3
:10631000811193C00E94720F90C0803291050CF0E1
:106320008CC0FC013197E930F10508F076C0E55BDF
:10633000FF4F0C94CD3A8091D902813011F482E064
:1063400010C0823029F41092D9021092E70265C081
:106350008091E702811104C081E08093E7025DC073
:1063600081E08093D90259C08091D8029EEF980FA6
:10637000923018F086568230C8F4C090D605D0907E
:10638000D705E090D805F090D905C701B6010E9465
:10639000111A082F87FD0AC00E944D0F282F30E0E8
:1063A00040E050E0C701B6010E94D919B3E04B1696
:1063B000510411F44FEF01C041E06091D605709196
:1063C000D7058091D8059091D9050E940D1B25C055
:1063D0008091FC028F5F863008F081E08093FC02A0
:1063E0006CEF72E086E591E00E94030C0E9465115B
:1063F00014C00E94F90E11C081E090E00E94EA12E0
:106400000CC081E090E00E94EA2407C00E9455067B
:1064100004C081E090E00E94B7120E9454240E94C0
:10642000250E6091D6057091D7058091D805909181
:10643000D9050E94FA170E942D110E94150D4816C9
:10644000590609F06CC16AE070E080E090E00E94BB
:106450003C2880E00E94F51FF0CFB090DB03BB200A
:1064600029F080911C018F3F31F40AC00E94920CE8
:10647000009741F4F6CF8091C603813009F05CC0EB
:1064800080E090E02091C503222329F097FF03C00C
:1064900021502093C5036091C5032091C403462F6A
:1064A00050E0EAE02E9F900111242150310942175B
:1064B000530734F4181619061CF46F5F6093C50374
:1064C0008091C5036AE00E94583AF82E8093E10259
:1064D000D0901C018D111BC68091C603813061F5DF
:1064E0000E9476280091C0031091C1032091C2033D
:1064F0003091C303061717072807390708F407C6A2
:106500001BC081E00E94F21C61E089E70E945F0FDE
:106510001092C6030E947628DC01CB018C509E4F5E
:10652000AF4FBF4F8093C0039093C103A093C203AA
:10653000B093C303F0921C0121E0E2128AC00E94D2
:106540002B2420911B01892B09F053C0213099F491
:106550000E947628DC01CB018C509E4FAF4FBF4F7D
:106560008093BB039093BC03A093BD03B093BE0381
:1065700010921B016EC00E9476280091BB031091FF
:10658000BC032091BD033091BE03061717072807EF
:10659000390708F05EC08091E1028093BA038981D7
:1065A0008093B9038D818093B80382E080930803C0
:1065B0001092BB031092BC031092BD031092BE0355
:1065C0001092E0021092DF021092DE028091060328
:1065D000811144C060E081E00E943F1A0E942D11A9
:1065E00080911E0190E062E0880F991F0E9493192C
:1065F00030C021112EC04090BB035090BC0360906E
:10660000BD037090BE03411451046104710409F18B
:10661000E0921B010E947628641575058605970592
:10662000C0F481E0B81201C080E08093DB0341E058
:10663000B41203C061E073E002C062EF72E081E077
:106640000E94901260E088EE93E00E9493190E94ED
:106650002D1180910803823009F054C00E94291E38
:106660008091DE0281114EC00E9476280091BB030A
:106670001091BC032091BD033091BE03AB01BC015E
:10668000401B510B620B730B80911F0190912001F5
:106690009C01220F331F820F931FA0E0B0E08417EC
:1066A0009507A607B70770F580910603811104C00E
:1066B00060E081E00E943F1A8091B80391E0980F5A
:1066C0009093B80390E08D5D9C4F0E942D0C0E942A
:1066D000BA1E9091B8038091B903891708F45BC57D
:1066E0000E9476286093BB037093BC038093BD0324
:1066F0009093BE038091DA02813021F41092DA0285
:106700000E942D110E94490D892B49F01092080317
:106710000E94651160E088EE93E00E9493198091D9
:106720002201882309F420C19924939455E0B52EC1
:1067300064E0A62E13E08091CB03823009F450C0B0
:1067400030F4882369F0813009F43EC001C18430FF
:1067500009F4ACC008F45EC0853009F4D7C0F8C0B5
:1067600080E00E94861D082E000C990B019703976C
:1067700020F080912101837031F081E00E94861D1C
:106780009092CB03E5C0C090E302D090E402E09089
:10679000E502F090E602C114D104E104F10409F429
:1067A0003CC50E947628C616D706E806F90608F00A
:1067B00034C51092E3021092E4021092E5021092A6
:1067C000E6020E94391929C58091210180FFB7C0D6
:1067D00084608093210180911F01909120010DC060
:1067E0008091210181FFB2C080911F019091200111
:1067F0009C01220F331F820F931FA0E0B0E0809313
:10680000C7039093C803A093C903B093CA0310931E
:10681000CB039EC080910603811126C080911E018A
:1068200090E062E0880F991F0E9493190E947628D9
:1068300020911D01AAE02A9F900111246901330FC4
:10684000EE08FF08DC01CB018C0D9D1DAE1DBF1DA8
:106850008093E3029093E402A093E502B093E602F2
:1068600061E081E00E943F1A0E947628C090C70331
:10687000D090C803E090C903F090CA03DC01CB01BB
:106880008C0D9D1DAE1DBF1D8093C7039093C80343
:10689000A093C903B093CA03809121018C7F809398
:1068A0002101A092CB030E94001E52C00E947628B4
:1068B000C090C703D090C803E090C903F090CA030A
:1068C000C616D706E806F906C8F40E94DA1D0E942B
:1068D000762820911F0130912001DC01CB01820F2D
:1068E000931FA11DB11D8093C7039093C803A0936C
:1068F000C903B093CA03B092CB032AC0809121018F
:1069000084FF26C081E00E94861D22C081E00E9493
:10691000861D0E947628C090C703D090C803E090DF
:10692000C903F090CA03C616D706E806F90680F434
:106930008091210182FF07C08A7F8093210182E03C
:106940008093CB0305C08D7F809321011092CB03F0
:1069500001E082E00E94F51F0111EDCE56C00E94B9
:10696000DA1D82E00E94F51F80E00E94861D8130C2
:10697000B9F580910603811126C080911E0190E037
:1069800062E0880F991F0E9493190E947628209137
:106990001D01BAE02B9F900111248901330F220BB6
:1069A000330BDC01CB01800F911FA21FB31F80931B
:1069B000E3029093E402A093E502B093E60261E063
:1069C00081E00E943F1A0E94001E80E00E94861D06
:1069D000813029F663E081E090E00E949319F5CFC1
:1069E000C090E302D090E402E090E502F090E6026D
:1069F000C114D104E104F10441F00E947628C616C6
:106A0000D706E806F90608F40AC480910603811146
:106A100036C180910803882329F08091DB038130FF
:106A200009F02DC180910503882309F44AC00E9412
:106A3000920C0091D6051091D7052091D805309180
:106A4000D90597FF15C0E091FC0244E0E49FF001F6
:106A50001124EC51FD4F80819181A281B381B90154
:106A6000A801481B590B6A0B7B0BDB01CA0112C042
:106A7000892BC1F0E091FC0254E0E59FF001112464
:106A8000EC51FD4F80819181A281B381800F911FD4
:106A9000A21FB31F8093D6059093D705A093D80566
:106AA000B093D9056091D6057091D7058091D8052E
:106AB0009091D905061717072807390709F0A6C0CE
:106AC000A9C080916201803129F48091C70580FFBF
:106AD00007C0A0C0843121F48091C70581FD9AC010
:106AE0000E94920C8C01892BF1F48091D00390913B
:106AF000D103892B09F48EC00E947628DC01CB01DA
:106B0000885E9340A109B1090091CC031091CD0397
:106B10002091CE033091CF03081719072A073B07AE
:106B200008F488C377C00E9476286093CC037093E2
:106B3000CD038093CE039093CF03101611061CF45F
:106B400021E030E002C02FEF3FEF8091D003909121
:106B5000D103820F931F9093D1038093D003889F1A
:106B60009001899F300D300D1124253031050CF432
:106B700051C00E9476281092D1031092D003C09089
:106B8000D605D090D705E090D805F090D905E091D2
:106B9000FC0264E0E69FF0011124EC51FD4F2081DE
:106BA000318142815381D8010E94ED3A6C0D7D1DE7
:106BB0008E1D9F1D6093D6057093D7058093D805D1
:106BC0009093D905A0E8CA16A6E9DA06A8E9EA066C
:106BD000F10458F46138B6E97B07B8E98B079105F1
:106BE000A8F021E02093E70211C0E0E8CE16E6E924
:106BF000DE06E8E9EE06F10449F06038F6E97F07C1
:106C0000F8E98F07910510F41092E7020E94FA1735
:106C10000E942D1180910803811131C00E947628B5
:106C2000DC01CB018A5F9109A109B1090091D70369
:106C30001091D8032091D9033091DA03081719076E
:106C40002A073B07E0F48091FF0283FF05C0809193
:106C5000FE02882309F4F3C281E090E00E947D0FD8
:106C600080910603882309F4F3C20E94762860937A
:106C7000D7037093D8038093D9039093DA0381E00C
:106C800090910603911101C080E00E94F51F809150
:106C9000040381110E9487060E947C030C94D92A68
:106CA00061E080E00E943F1A62E370E080E090E0E3
:106CB0000E943C280C94F72A0E9439190C94012B4D
:106CC000C80101970D3F1F4FCCF46091D60570911C
:106CD000D7058091D8059091D9054FEF09C06091F3
:106CE000D6057091D7058091D8059091D90541E0DE
:106CF0000E940D1B00E010E00C94AC2C8C010C9455
:106D0000AC2C10929A021092990210929802609103
:106D1000D6057091D7058091D8059091D9050E942C
:106D2000FA170E94250E0C945F2D10929702609125
:106D3000D6057091D7058091D8059091D9050E940C
:106D4000FA1712C063E172E081E00E94901260E0E5
:106D500084EF91E00E9493198FEF80931C0181E0F2
:106D6000809308030E942D111092C805CBCA902E63
:106D70000C94322E10929B0260E081E00E943F1A38
:106D800069817A818B819C810E94C81760E882E1C9
:106D90000E94550D63E171E082E20E947E256BE066
:106DA00071E08AE30E947E2560E881EB0E94550D28
:106DB0006FE682E10E94550D60910A016B7F60933E
:106DC0000A0183E00E94550D61E082E00E94A42543
:106DD00061E173E078876F830E9476286B017C0104
:106DE0006093090370930A0380930B0390930C0341
:106DF000EF81F8854191F887EF832D813E81429F95
:106E0000C001439F900D112480900D0390900E03BC
:106E1000A0900F03B0901003880E991EA11CB11C06
:106E2000692D88E20E94550D682D89E20E94550D5A
:106E300046015701FBEA8F0EF2E09F1EA11CB11C18
:106E40000E947628681579058A059B05C8F34F814D
:106E50005885435B534009F0BFCF60E082E00E9459
:106E6000A4250E94391999249A940C94322EC09228
:106E70006902D0926A02E0926B02F0926C0271C9D0
:106E80000E94920C181619060CF5809169029091D7
:106E90006A02A0916B02B0916C02825D9D4DAF4F72
:106EA000BF4F8093690290936A02A0936B02B093E4
:106EB0006C028091650290916602A0916702B09188
:106EC000680288589F4FAF4FBF4F23C0892B09F4EA
:106ED000B0C88091690290916A02A0916B02B09152
:106EE0006C028E529242A109B1098093690290937B
:106EF0006A02A0936B02B0936C028091650290913C
:106F00006602A0916702B091680288579109A109B1
:106F1000B1098093650290936602A0936702B093D3
:106F200068028091690290916A02A0916B02B0910F
:106F30006C0280549F48A84DBB4C809306019093EF
:106F40000701A0930801B093090140916502509197
:106F50006602609167027091680280E00E94700D85
:106F60002EC80E94920C1816190664F480916502CE
:106F700090916602A0916702B09168020597A109FD
:106F8000B1090EC0892B09F490C8809165029091D7
:106F90006602A0916702B09168020596A11DB11D1D
:106FA0008093650290936602A0936702B093680293
:106FB000409165025091660260916702709168028B
:106FC00080E00E94700D6091650270916602809170
:106FD0006702909168020E94701180E00E94F51F84
:106FE00064E670E080E090E00E943C285EC80E9469
:106FF0002B24892B51F462E371E080E00E9490120F
:1070000065E672E088E090E016C0C0926502D0921A
:107010006602E0926702F09268021DC00E942B2473
:10702000892B89F466E071E080E00E94901261E6AD
:1070300072E08CEF90E00E94650B60E088EE93E0D8
:107040000E94931908C0C0926102D0926202E0923D
:107050006302F09264028091D902811109C04091CB
:10706000650250916602609167027091680209C0E2
:1070700040916102509162026091630270916402DA
:1070800080E00E94700D6FC80E94920C18161906BD
:1070900064F48091610290916202A0916302B091C8
:1070A00064020597A109B1090EC0892B09F434C8FF
:1070B0008091610290916202A0916302B09164029A
:1070C0000596A11DB11D8093610290936202A09369
:1070D0006302B09364024091610250916202609138
:1070E00063027091640280E00E94700D6091610201
:1070F0007091620280916302909164020E9470110B
:1071000060E084E690E00E9493190C948C300F2D7F
:1071100010E0000F111FBE016B5F7F4FC8018D5D36
:107120009C4F0E94D30BBE016F5F7F4FC8018C5DE7
:107130009C4F0E94D30BFD100EC08091BF038F5F48
:107140008093BF0390E0298130E04D81241B3109F9
:107150002817390714F41092BF036F2D87E70E9498
:107160005F0FC980D12CF5E1CF0ED11C0D8110E04D
:107170000B5E1F4F81E60E941B0CC016D1060CF45B
:10718000C0C9C801825F9C4F0E942D0C0E94F31B56
:107190000F5F1F4FF2CFF090DF02FF2079F10091D7
:1071A000DB020093BA038091DC028093DB028091C2
:1071B000DD028093DC0210E0000F111FBE016B5F47
:1071C0007F4FC8018D5D9C4F0E94D30BBE016F5F46
:1071D0007F4FC8018C5D9C4F0E94D30B89818093A7
:1071E000B9038D818093B803FA94F092DF0280E2B4
:1071F0000E94BA1E81E08093DA0272CA81E0809315
:10720000080380911D0162E05AE0859FC0011124AE
:107210000E9493190E94391963CA00E09ACB109218
:10722000E3021092E4021092E5021092E6020E943C
:107230003919EBCB1092D1031092D003EBCC809193
:10724000D2038F5F8093D20384300CF05CC004CDF6
:1072500080910503811109CD4091000350910103F4
:1072600060910203709103038091D6059091D70538
:10727000A091D805B091D905481759076A077B072F
:10728000D9F00E9476286093D3037093D40380933F
:10729000D5039093D6038091D6059091D705A09100
:1072A000D805B091D9058093000390930103A09372
:1072B0000203B0930303D9CCC090D303D090D4037E
:1072C000E090D503F090D603C114D104E104F10499
:1072D00009F4CBCC0E947628DC01CB018C199D09E6
:1072E000AE09BF0981319742A105B10508F4BDCCB3
:1072F0000E9454241092D3031092D4031092D50309
:107300001092D603B2CC89E590E00E942F0C8093B6
:10731000FD021092D203A0CC812F662D0E94583A14
:10732000082F0C94552EE1EEF5E01382128288EEC0
:1073300093E0A0E0B0E084839583A683B78324E93B
:1073400031E03183208325EC30E03587248724EC3D
:1073500030E03787268720EC30E0318B208B21EC22
:1073600030E0338B228B22EC30E0358B248B26EC03
:1073700030E0378B268B118E128E138E148EEEE733
:10738000F6E01382128284839583A683B78386EA0C
:1073900091E0918380830895BB274A3031F499238B
:1073A00022F4BDE2909581959F4F0C94093ABB273A
:1073B0002A3051F4992342F4BDE29095809570955E
:1073C00061957F4F8F4F9F4F0C94E739BB27FA0190
:1073D000A62F6217710581059105330B30FB66F00E
:1073E000AA27660F771F881F991FAA1FA21710F0E0
:1073F000A21B63953850A9F7A05DAA3308F0A95DD8
:10740000A19336F7B111B1931082CA010C94223ABC
:10741000BB27FB015527AA27880F991FAA1FA4176E
:1074200010F0A41B83955051B9F7A05DAA3308F062
:10743000A95DA193009779F7B111B1931192CB0196
:107440000C94223ADC01FC01672F71917723E1F75C
:10745000329704C07C916D9370836291AE17BF0721
:10746000C8F30895F999FECF92BD81BDF89A992786
:1074700080B50895262FF999FECF1FBA92BD81BD20
:1074800020BD0FB6F894FA9AF99A0FBE01960895A6
:10749000DB018F939F930E94E23ABF91AF91A29F2D
:1074A000800D911DA39F900DB29F900D1124089502
:1074B000991B79E004C0991F961708F0961B881F46
:1074C0007A95C9F780950895AA1BBB1B51E107C0A7
:1074D000AA1FBB1FA617B70710F0A61BB70B881F64
:1074E000991F5A95A9F780959095BC01CD010895F3
:1074F00097FB072E16F4009407D077FD09D00E9461
:10750000643A07FC05D03EF4909581959F4F08950D
:10751000709561957F4F0895A1E21A2EAA1BBB1B9F
:10752000FD010DC0AA1FBB1FEE1FFF1FA217B3074F
:10753000E407F50720F0A21BB30BE40BF50B661F65
:10754000771F881F991F1A9469F760957095809529
:1075500090959B01AC01BD01CF010895052E97FBCD
:107560001EF400940E94C53A57FD07D00E948C3A41
:1075700007FC03D04EF40C94C53A509540953095D5
:1075800021953F4F4F4F5F4F08959095809570958F
:1075900061957F4F8F4F9F4F0895EE0FFF1F05900E
:1075A000F491E02D0994A29FB001B39FC001A39F65
:1075B000700D811D1124911DB29F700D811D11242C
:1075C000911D08950E94D33AA59F900DB49F900DF0
:1075D000A49F800D911D11240895B7FF0C94E23AE9
:1075E0000E94E23A821B930B089581E090E0F894A8
:1075F0000C942C3BDC0101C06D9341505040E0F7EE
:107600000895FB01DC010D900020E9F7119701902E
:107610000D920020E1F70895FB01DC018D910190AE
:1076200080190110D9F3990B0895FB01DC01019039
:107630000D920020E1F70895FB01DC010D90002080
:10764000E9F711974150504028F0019000200D9229
:0C765000C9F708951C920895F894FFCF2C
:10765C00FF0120030000C0702734FF000100000070
:10766C00000000FFFE00000000000001FF3C32643F
:10767C00001001E80364000A00706D2E63302E7652
:10768C00616C3D00FFFFFFFFFFFF000100000000E9
:10769C0000000300706D2E73302E7478743D2270D0
:1076AC006D2E76302E76616C3D01B0196D00C0AC3C
:1076BC00D80010FF0E0F1011141530313233343541
:1076CC0036373839616263646566706D2E73682E67
:1076DC007478743D220303030102040507090A0BA5
:1076EC00000000000D037A02A4025A03D502B30273
:1076FC00C702000000001304E6034304BA03DE03D0
:10770C00CA03BB032B76312E3230300054756E65B4
:10771C0020537465703A00204C534220555342203C
:10772C0043574C204357550049465300415454008D
:10773C0043573A0057504D204368616E67653F00D0
:10774C0057504D0053454E443A20005054542D3E52
:10775C00200063616C3A00546F6E650044656C6187
:10776C00790020535420204941202049420045787B
:10777C0069743F00203A0053617665642046726557
:10778C007175656E6379004348002E005072657305
:0A779C00732C207365742000220096
:00000001FF
